:100000000C9466000C9487000C9487000C94870075
:100010000C9487000C9487000C9487000C94870044
:100020000C9487000C9487000C9487000C94870034
:100030000C9487000C9487000C9487000C94870024
:100040000C9487000C9487000C9487000C94870014
:100050000C9487000C9458030C9487000C94870030
:100060000C9487000C9468130C9487000C94870000
:100070000C9487000C9487000C9487000C948700E4
:100080000C94A0000C9487000C9487000C948700BB
:100090000C94621B0C9487000C9487000C948700CE
:1000A0000C9487000C9487000C9487000C948700B4
:1000B0000C9487000C9487000C9487000C948700A4
:1000C0000C9487000C9487000C94870011241FBEA9
:1000D000CFEFD1E2DEBFCDBF00E00CBF14E0A0E067
:1000E000B2E0E6E8FAE900E00BBF02C007900D922B
:1000F000A434B107D9F717E0A4E4B4E001C01D921D
:10010000AC33B107E1F70E94050D0C94414D0C94FE
:1001100000001092550410924A0480914A04809382
:100120004904809149048093480480914804809355
:10013000470410924B0410925804109259040895E9
:100140001F920F920FB60F9211240F900FBE0F90B7
:100150001F901895EEE6F0E080818260808383E056
:1001600084BD85BD8AEF87BD08951092900088E018
:10017000809391008BE09AE190939900809398008E
:10018000109295001092940082E08093710008957F
:100190000895089580917100817008959B01AC01CC
:1001A000CA01AA27BB27BC01892B79F0687F672B7E
:1001B00059F483E056954795379527958A95D1F759
:1001C0003093AF042093AE0408953093AF0420938E
:1001D000AE0408958091AC04982F929596959695CB
:1001E0009370282F221F2227221F9227282F229523
:1001F0002F709227282F2695269592279170880F89
:10020000892B8093AC04089590939E0480939D0461
:1002100085EB9BE39093B6048093B50483E393E16D
:100220009093BC048093BB0485E694ED9093B10455
:100230008093B004089580919D0490919E04AC0138
:10024000440F452F441F550B51954827592760915E
:10025000B5047091B60470939E0460939D048091E0
:10026000BB049091BC049093B6048093B504209194
:10027000B0043091B1043093BC042093BB04C90195
:100280000024969587950794969587950794982FBF
:10029000802D8227932784279527542F4427529512
:1002A000550F507E842795279093B1048093B00416
:1002B000660F771F6F5F7F4F869F9001879F300D7E
:1002C000969F300D1124C9010895FC019081992356
:1002D00051F08091C80085FFFCCF9093CE003196FD
:1002E00090819923B1F708951F93CF93DF93182F2F
:1002F000492FE0E1F7E2C0E0D0E0812F942FBF0169
:100300000E94F84C9B016115710589F5812F942F8E
:10031000BF010E94F84C182F492FCF016AE070E00E
:100320000E94F84CFB012196C430D10531F730977B
:10033000A1F18091C80085FFFCCF812F942FBF01D0
:100340000E94F84C605D6093CE00CF016AE070E0DF
:100350000E94F84C9B0161157105F9F0812F942FD3
:10036000BF010E94F84C182F492FF901E2CF80916C
:10037000C80085FFFCCF822F805D8093CE00812F47
:10038000942FBF010E94F84C182F492FCF016AE02B
:1003900070E00E94F84CFB01CACFDF91CF911F9112
:1003A0000895982F9F709A3040F48091C80085FF7F
:1003B000FCCF905D9093CE0008958091C80085FF9A
:1003C000FCCF995C9093CE000895CF93DF93EC011E
:1003D000892F992782958F700097C1F48D2F9927C7
:1003E000009789F4CE01929582958F7089279F702E
:1003F0008927009711F00E94D1018C2F0E94D10112
:10040000DF91CF9108950E94D101ECCF0E94D101DC
:10041000E5CF982F8091C80085FFFCCF9093CE0048
:1004200080E090E008952091C800332727FD3095A3
:100430002227330F221F3327C90108958091C80056
:1004400087FFFCCF8091CE0090E008959C018FEF54
:100450008093A20493E0283E390768F580939F04B7
:100460008093A00424363105D8F0C90164E670E019
:100470000E94F84C60939F04C9016AE070E00E94FA
:10048000F84CCB016AE070E00E94F84C8093A00425
:10049000C9016AE070E00E94F84C8093A1040895BD
:1004A0002A30310548F7C9016AE070E00E94F84C33
:1004B0008093A104089510929F041092A0041092BA
:1004C000A104089590914C04936090934C04809300
:1004D0004D04089580914C04836080934C040895EA
:1004E000F999FECF92BD81BDF89A30B5F999FECF4A
:1004F000019692BD81BDF89A20B5932F80E030E03F
:10050000282B392BC9010895F999FECF92BD81BDE1
:10051000F89A80B50895F999FECF92BD81BD60BD6E
:10052000F894FA9AF99A78940895FF920F931F938A
:100530008C01F62E672F0E948B02C80101966F2D49
:100540000E948B021F910F91FF9008958091C90026
:1005500088618093C90083E38093CC001092CD0022
:100560008091C80087FD34C08091C9008068809365
:10057000C9008091C10088698093C1008FE1809398
:10058000C4001092C50090EC91B98CE382B987E366
:1005900084B995B99FEF97B988EF8AB98BE08BB989
:1005A00082E08DB99EB910BA91BB88E183BB87EE1A
:1005B00084BB8DB581608DBD81E58CBD0895809132
:1005C000CE008AE00E94CC0F8091C80087FFCCCF7C
:1005D0008091C80087FDF3CF8091C80087FFF8CFD6
:1005E000EECFEF92FF920F931F93CF93DF93EC0127
:1005F00081E0CD32D80708F440C0CCE2D1E07E01E2
:1006000000E010E08091990490919A048C179D0766
:1006100019F0CE010E941D1BD0939A04C093990437
:10062000D093AB04C093AA046091090270910A02AE
:1006300080910B0290910C02A80197010E941F4D1E
:100640006FEF7FEF8FEF9FEF0E941F4DCA01B9013F
:1006500028EE33E040E050E00E94CD4C6093A604C9
:100660007093A7048093A8049093A904DF91CF917D
:100670001F910F91FF90EF900895C431D10508F0BC
:10068000BECFC4E1D0E054E1E52EF12C012D112DB7
:10069000B9CF85E090E00E9470020E94F102809143
:1006A000990490919A049093B3048093B2040895AE
:1006B0001F920F920FB60F920BB60F9211242F9329
:1006C0003F934F935F936F937F938F939F93AF93DA
:1006D000BF93EF93FF9340B1427090B18091B90402
:1006E000481749F1892F8170442309F4D8C0882321
:1006F00009F4D8C09FEF809101048823D1F0809144
:100700005304882309F4FAC0913009F017C180918D
:10071000AA049091AB0407969093AB048093AA042B
:100720008D52914030F08CE291E09093AB04809335
:10073000AA044093B904809169048F3F29F0809105
:1007400069048F5F8093690480916A048F3F29F068
:1007500080916A048F5F80936A04809178049091FD
:1007600079048F5F9F4F49F08091780490917904CC
:10077000019690937904809378048091560488239D
:1007800051F0809156048150809356048091560414
:10079000882309F49AC080919404909195048F5F06
:1007A0009F4F49F080919404909195040196909305
:1007B00095048093940480914404823009F487C0A6
:1007C000813009F471C0882309F056C0809101027C
:1007D00090910202A0910302B0910402809305025D
:1007E00090930602A0930702B093080220910102A1
:1007F0003091020240910302509104028091A604BC
:100800009091A704A091A804B091A904820F931F0E
:10081000A41FB51F8093010290930202A0930302CC
:10082000B093040220910102309102024091030230
:10083000509104028091050290910602A091070256
:10084000B0910802281739074A075B07A8F480917E
:1008500055048F5F80935504809155048170809377
:100860005504809154048F5F809354048091AA04AE
:100870009091AB040E94F102FF91EF91BF91AF9173
:100880009F918F917F916F915F914F913F912F91A8
:100890000F900BBE0F900FBE0F901F9018958823DE
:1008A00009F428CF91E027CF99B19295917080916A
:1008B0006704981709F39093550490936704809107
:1008C00054048F5F80935404D7CFA49864CF809151
:1008D000630490916404892B79F280916304909170
:1008E000640401979093640480936304809163048B
:1008F00090916404892B09F0BFCFE1CF292F3327D2
:1009000027FD30958091AA049091AB04280F391FE0
:100910003093AB042093AA0481E02D32380708F00D
:1009200002CF2431310508F004CF84E190E09093A8
:10093000AB048093AA044093B904FDCE9F3F09F015
:10094000F8CE8091AA049091AB0407979093AB04E2
:100950008093AA04449708F0ECCEE7CFCF92DF92C1
:10096000EF92FF920F931F93CF93DF93F8948091B0
:100970004404813009F4C7C480919004813009F4A3
:10098000DFC2809147048C3060F010924704809160
:1009900048048F5F80934804809149048F5F80935F
:1009A000490480914904882341F08091490490E0F2
:1009B00083709070892B09F45CC280914A0488305E
:1009C00038F010924A0480914404882309F430C21C
:1009D000809149048F7080934904909148048091DC
:1009E00000029817C0F01092480480914B048F5F6A
:1009F00080934B0490914B048091BA04981708F0AF
:100A000014C280914C04826080934C048091500405
:100A100081608093500480913607882329F4809167
:100A20004804882309F4F7C180914804882329F4F5
:100A300080919004823009F4A3C29091580480916F
:100A4000B404981710F01092580480913607882348
:100A500029F080915804882309F411C28091F80488
:100A60008C3009F415C280914404882309F005C133
:100A7000909162048091FF03981710F01092620425
:100A80008091620480FFF3C05C9880919104209172
:100A9000FF034091FF0390E030E0240F311D8217E7
:100AA000930714F010929104E091FF03E695E69508
:100AB000E69520915A0490919104E150F0E0EE0FF8
:100AC000FF1FEE0FFF1FE20FF11DE35FFD4F80815F
:100AD000891709F4F9C1DD248091FF03869590916F
:100AE000AD04899F902D112480915904891710F02D
:100AF0001092590480913607882349F08091590457
:100B0000882309F4A39A9695891709F449C280911C
:100B1000F804873009F4D3C0883008F4C8C08B309B
:100B200009F4CDC08C3008F43DC28C3009F46DC39B
:100B30008D3009F4C4C080919004823009F4FBC365
:100B400080913607882321F082E0D81609F4FEC38D
:100B500080913607882309F403C280917D048F7049
:100B600080937D048091490490E083709070029797
:100B70000CF4F2C185E20E94361780917D0490E06A
:100B80008370907002970CF4E4C18FEF809375042A
:100B900080918604882309F0A3C180918F04882363
:100BA00071F080914D04882351F08091B704813019
:100BB00009F42BC28091B704882309F416C28091EE
:100BC0004E04813009F4E2C3823009F4C3C380913A
:100BD0005304882349F080914404882329F48091A8
:100BE0000104882309F021C20E940D19DD2031F093
:100BF000809145048F5F81708093450480919104BA
:100C00008F5F8093910480912A078F5F80932A07DA
:100C1000809147048F5F80934704809162048F5FC7
:100C200080936204809158048F5F80935804809170
:100C300059048F5F8093590420912A078091FF0304
:100C400030E086958695869548E1849FC001112401
:100C50002817390714F010922A077894DF91CF9162
:100C60001F910F91FF90EF90DF90CF9008955C9AC5
:100C700088EF0E94D71080914404813009F419C193
:100C8000823009F002CF809155048F5F8093550424
:100C90008091550481708093550480915504882378
:100CA00009F4F2CE5C9A88EF0E94D710EECE813024
:100CB00008F441CF843018F0853009F03CCF81E052
:100CC000D81609F4E8C1E2E0DE1609F034CF8091CD
:100CD0007D048F5F80937D0480913607882309F41B
:100CE00094C08091BD05882309F510922A07809150
:100CF000C105882349F480912C07882329F080912D
:100D00008604882309F03BC68091450660918D06D4
:100D1000680F8091D1069091D2060E94022D109208
:100D20007D0480918104882309F447C58091BD0525
:100D3000E091D106F091D206E80FF11D80818093F9
:100D400098048091A5048093A304809198048074F2
:100D50008093A50480918604882309F0C4C48091FF
:100D600098048F708F3009F41EC5809198048F709D
:100D70008F3029F1809198040E94262D0091D7068A
:100D8000080F1091980410786091A304802F412FD0
:100D90000E94871E112309F00EC580E0902F935FFB
:100DA000982B80915104981751F0809151048093B1
:100DB000520490935104809151040E948B108091B1
:100DC000F804833009F47EC48091F8048730E9F494
:100DD00080914E04882309F0C4C58091A4059091A8
:100DE000A505E091B605F0E0EE0FFF1FEB5EFD4FAD
:100DF0006081718182959295907F9827807F982756
:100E00000E94F84C862F0E94E61780914C04816066
:100E100080934C0490CE80919004823009F004CEEF
:100E2000109290040E944D36FFCD10924B04E9CDF4
:100E30002091990430919A048091B2049091B30466
:100E40002817390709F4C4CD80913607882309F0A3
:100E5000BFCD85E20E94FE166091990470919A04BC
:100E60007093B3046093B20485E090E00E94950211
:100E7000AFCD80914A048F5F80934A049ECDA49A9F
:100E800085E0809356048091F8048C3009F0EBCD16
:100E90008091500480FF0AC080913607882309F0B2
:100EA0007EC280915E04882309F083C310925004AF
:100EB000DACD80915504882309F4E7CD88EF0E94AC
:100EC000D71080914404DCCE2F5F237020935A0406
:100ED00080914504882309F450C0DD24D394FCCDCF
:100EE0008CE20E94262D982F80917D048111945FC1
:100EF00080912A07882341F480918704882309F48C
:100F0000A0C383E20E94FE1680912A07843009F074
:100F100044CE80918704882379F4809184048230C0
:100F200008F4B2C3809149060E94262D40914906DB
:100F3000407860E00E94871E83E20E9436172DCE23
:100F400080913607882381F00E942331109290040B
:100F500018CD109275041CCE85E20E94FE160DCEAF
:100F600081E20E943617F9CD0E944D3680914404EB
:100F7000882361F70E948900E9CF52E0D52EACCDDD
:100F80008091F804853009F458CD10925A041092DB
:100F90009104109245041092BD05109290044DCD1D
:100FA000A398B5CD883009F0C6CDF1E0DF1609F47D
:100FB0004EC382E0D81609F0BECD8091970480938D
:100FC000460480919604809397040E94EA008093DF
:100FD0009604809197048F7360E040E00E94871E22
:100FE000809197040E948B10A6CD80914C0480FFC5
:100FF000E6CD80914C048E7F80934C040E94C217F2
:101000008091BD050E94D017DACD80914C0481FFFC
:10101000D1CD80914C048D7F80934C040E94C217E7
:1010200080914B040E94D017C5CD0E94C2176091D9
:10103000990470919A04603A710508F489C2603A83
:10104000710509F436C380E090E02EE030E040E026
:1010500050E00E94CD4C685E7E4F8F4F9F4F28E13D
:1010600031E040E050E00E941F4D022F293008F48B
:1010700080C418E0812F0E94D0171F5F1017D0F393
:10108000003108F0B1CD102F812F0E94DB171F5FB8
:101090001031D0F3A9CD8091C1058F5F8093C10538
:1010A00080913607882309F446CD8091BD058F5F76
:1010B0008093BD059091BD0580910004981710F0B4
:1010C0001092BD058091BD05882309F06EC0809106
:1010D000F804833009F49AC210E08091F804873054
:1010E00009F425C381E00E94D12C80918D068F5F89
:1010F00080938D06C0908D0690918D0680914B0651
:10110000981708F443C080918104882319F481E082
:1011100080938E048091F804813009F469C3809132
:10112000F804823009F460C382E00E94D12C10924E
:10113000C10580918604882369F08091840480939E
:101140002C0780912C07882329F01092840481E0D9
:101150008093BB0510928D068091F804833009F4CA
:101160009AC38091F804873009F459C380914C06E2
:10117000882309F040C3909129078091BC059817F6
:1011800029F080918104823008F42DC480918D066D
:1011900090E082959295907F9827807F982781573D
:1011A000994F9093D2068093D1068091860488232C
:1011B00009F0C1CC8091BD05E091D106F091D20635
:1011C000E80FF11D808180939804809198048F70BE
:1011D0008F3009F4A9C28091A5040E949E1E8091BF
:1011E0005204882309F099C28091A504882309F04C
:1011F000A2CC80915104882309F49DCC80915104A4
:101200000E94B1101092510496CC0E94C217809196
:10121000500480FD14C180915E04882309F009C147
:10122000E1E0DE1609F40FC1F2E0DF1609F083CC2D
:1012300080917D048F5F80937D04809136078823A1
:1012400009F479CCE0918D06F0E0ED52F94F808100
:1012500084FD25C28CE08093FF038091BD05E09161
:10126000D106F091D206E80FF11D80818093980499
:101270008091A5048093A304809198048074809346
:10128000A504809198048F708F3009F43BC280913F
:1012900098048F708F3071F0809198040E94262DF1
:1012A0009091D7066091A304409198044078890FEB
:1012B0000E94871E80914F04982F92959F70909363
:1012C000E806982F977090934506869586958695A3
:1012D00081708093290780912907882309F0D8C15C
:1012E00088E00E94FE1681E00E9436170E94B61820
:1012F000809145068F5F0E94561880913607817055
:101300008093360718CC0E940E14882339F0809100
:101310008F04882309F0ADC10E9489000E94201427
:10132000882309F429CB80918F04882309F424CBE6
:101330000E94233121CB81E20E943617809147041D
:1013400090E083709070892B09F007CC81E20E94B5
:10135000FE1603CC0E94B41A90919F04892F8150ED
:10136000823008F482C19091A0048091A104981762
:1013700009F4D6C0992309F072C18091490480FD17
:1013800026CC8091A1040E94A91A21CC0E94B41AF3
:101390008091490480FFD0C080914E0415CC80918B
:1013A0003607823008F482CD80915E04882329F4C8
:1013B0008091A805882309F479CD80915F048093FA
:1013C0004F0490918D069F5F90938D0690918D06AE
:1013D000917090938D0660918D0670E06295729584
:1013E000707F7627607F76276157794F7093D2069A
:1013F0006093D10690918D06C92FD0E00E946C2F8A
:10140000CD52D94F8883E0918D06F0E0ED52F94F2F
:1014100080818F708F5F80930004E0918D06F0E0F3
:10142000ED52F94F808184FD1EC18CE08093FF0353
:101430003DCD80915E0481500E94D017F1CE8FE0A7
:101440000E94D017E8CE80913607882309F473CB29
:101450008091BD058F5F8093BD0580915E048823D8
:1014600009F40AC190915F0480914F048917D1F16A
:10147000F0908D06F394FE220F2D10E0E801C29546
:10148000D295D07FDC27C07FDC27C157D94F809110
:101490005F04BE010E946C2F0D52194FF80180832A
:1014A000E0918D06F0E0ED52F94F2081F801808146
:1014B00090E030E08227932784FD14C080915F0480
:1014C00080934F04F0928D06E0918D06F0E0ED528E
:1014D000F94F80818F708F5F80930004D093D20684
:1014E000C093D1068091BD05609100040E94EC4C30
:1014F0009093BD058091BD05E091D106F091D20693
:10150000E80FF11D808180939804809198048F707A
:101510008F3009F4C6C08091A5040E949E1E0BCB9B
:101520008091490482FD04C08091490480FD4FCB25
:10153000892F0E94A91A4BCBE0914904E695F0E06F
:10154000E370F070E156FB4F80810E94A91A24CF0E
:1015500080E090E02EE030E040E050E00E94CD4C92
:101560006E5070408040904028E131E040E050E013
:101570000E941F4D022F222309F434C110E0812F55
:101580000E94DB171F5F1017D0F3083008F028C146
:10159000102F812F0E94D0171F5F1830D0F3103109
:1015A00008F022CB812F0E94DB171F5F1031D0F390
:1015B0001BCB80915F0480934F040E944D36809135
:1015C0004404882309F4A6C010925A0480918D0621
:1015D0008F5F80938D0680918D06817080938D063C
:1015E00060918D0670E062957295707F7627607FBE
:1015F00076276157794F7093D2066093D106809118
:101600008D06C82FD0E080914F04F8CE8091A405BC
:101610009091A50501969093A5058093A40520912E
:10162000A4053091A5058091AF059091B0052817CC
:10163000390708F451CD1092A5051092A40511E0C8
:101640004CCD892F60E040E00E94871E5ACC80E09C
:101650000E949E1E809197040E94B1106CCA892F2F
:101660000E94A91A8ACE80E1E1CE865F0E94A91A63
:101670007ACE0E944D3650CE8091A805882309F07D
:1016800031CF0E9423312ECF80E00E949E1E54CC89
:1016900088E00E94361781E00E94FE1627CE80E186
:1016A000DACD8091A504882309F096C01092A50494
:1016B00032CF0E94C21787E00E94D01788E00E94B4
:1016C000D01792CA80914E04882309F042C18091BC
:1016D000B505882309F478CB0E94ED188091D706D0
:1016E0000E94C41871CB8091450660914B064091D1
:1016F000BE0520914C060091C205E090BC050E94F9
:10170000FC195DCB809198048F708093980410929F
:10171000A504BDCD0E94890057CF809152040E943C
:10172000B1101092520460CD1092A50454CD809156
:101730007C04813009F0D6CC609129078091450660
:1017400040918D062091D706480F8CEA95E00E94C3
:1017500008208091B6056091A4057091A50540917F
:10176000AC050E94B7218091A4059091A505019632
:101770009093A5058093A405E091B6052091A4055A
:101780003091A505F0E0EE0FFF1FEB5EFD4F80816D
:1017900091812817390708F4A5CC10927C0483E2C4
:1017A0000E9436179FCC809198048F708093980484
:1017B0001092A504DACA80E8F1CA809145066091CA
:1017C0004B064091BE0520914C060091C205E09069
:1017D000BC050E94FC19AACA81E00E949E1E66CF29
:1017E000102FDDCE10E0D5CE81E080938E049CCC0E
:1017F00080938E0494CC0E94BE2C80918104823010
:1018000008F0C4CC8091E806609129074091450614
:1018100020914B060FE816E00E94C92FB7CC8091AB
:101820007C04813009F0A2CC8091A8058823B9F00E
:1018300010927C041092A8058091B6056091A405D1
:101840007091A5050E948E218091B6050E941A22F2
:101850009093B0058093AF0583E20E943617809184
:10186000A905882309F482CC1092A9058091B605B8
:101870006091A4057091A5056C190E947E2180914C
:10188000B6050E9411229093B8058093B70580E0B9
:101890000E9436176BCC8091A805882309F098C068
:1018A0008091A905882309F466C01092A5051092BD
:1018B000A4058091F3048093B6058091B6050E943B
:1018C0001A229093B0058093AF058091B6050E94CF
:1018D00011229093B8058093B7052091B7053091F8
:1018E000B8058091AF059091B0052817390720F011
:1018F0001092B8051092B7058091A905882309F0C8
:1019000059C08091B6056091A4057091A5050E940B
:101910006B228093AC058091B6056091AC0544E0E4
:1019200056E02CEB35E00EEB15E090EDE92E96E05D
:10193000F92E0E94E81F81E080934C068091D0062A
:101940008D3010F01092D0068091D0068093D7068B
:1019500008CC8091A4059091A50501960E942602CD
:10196000B6CE8091A4059091A50501960E9426020D
:1019700034CA18E089CB112309F4BECF96CF81E099
:101980000E949E1E80E00E949E1E60914B068FE882
:1019900096E049EE56E023EC35E00E94312E10929D
:1019A00086048AE00E94422D1092A50482E00E94E3
:1019B000CC0FAAC91092A9058091B7059091B805DE
:1019C0009093A5058093A40580E00E94361799CFD7
:1019D0001092A8051092A5051092A40583E20E941A
:1019E000361711E05DCF8091BC05809329070ACF9F
:1019F00007C0809154048150809354040E94AE0427
:101A0000809154048823A9F70895AF92BF92CF9292
:101A1000DF92EF92FF920F931F93DF93CF93CDB797
:101A2000DEB760970FB6F894DEBF0FBECDBF0E9441
:101A3000A6020E94490380916E00826080936E002E
:101A400083E084BD85BD8AEF87BD8FE896E09093E3
:101A5000D2068093D106F999FECF82E090E092BD44
:101A600081BDF89A80B5982F937090934404829525
:101A7000817080938704F999FECF87E090E092BD52
:101A800081BDF89A80B5882311F0813208F080E199
:101A900080930002F999FECF83E090E092BD81BD72
:101AA000F89A80B58F708093D004F999FECF84E0C6
:101AB00090E092BD81BDF89A80B58F708093BD048F
:101AC00088E090E00E9470028093AC042091990419
:101AD00030919A04280F391F30939E0420939D045F
:101AE00085EB9BE39093B6048093B50483E393E185
:101AF0009093BC048093BB0485E694ED9093B1046D
:101B00008093B0040E941B010E941B010E941B01D4
:101B1000BC0188E090E00E949502F999FECF8AE02E
:101B200090E092BD81BDF89A90B5892F8F70809317
:101B3000B7048091B704833010F01092B7049295E7
:101B40009F709F5F9093BA048091BA04823018F41A
:101B500082E08093BA04F999FECF8DE090E092BDC7
:101B600081BDF89A60B5862F8C59893C08F437C13D
:101B700060ED72E183E190E0F89460930902709364
:101B80000A0280930B0290930C02F999FECF8EE02B
:101B900090E092BD81BDF89A40B5493008F416C175
:101BA00042E08CE08093B4044093AD04F999FECFF9
:101BB0008FE090E092BD81BDF89A80B5853008F045
:101BC00080E080935B040E94C530789400E010E0D0
:101BD0001DC08091FD040E94D0170E940D19C801FC
:101BE000849668E270E00E940C4D0E94A31A0E9445
:101BF000361780E10E94CC0FC80187709070892B46
:101C000069F00F5F1F4F0C32110579F0083208F7A9
:101C1000802F0E94A31A0E94FE16DBCF0E944C1652
:101C20000F5F1F4F0C32110589F70E94AD170E94FC
:101C30000D190E944C1680E00E948714882331F011
:101C400083E00E948714882309F022C183E00E9468
:101C50008714882309F0D3C08091FD048093E8069F
:101C6000109229071092BC051092450681E08093DE
:101C70004B0610924C068091E8066091290740912E
:101C8000450620914B060FE816E00E94C92F60918F
:101C90004506C8010E94022D0E948D2C0E944C1600
:101CA00080914C04836080934C0410924D04809189
:101CB000F804873009F487C08830B0F5823009F421
:101CC0005EC0833008F045C0882309F452C08130DB
:101CD00009F452C00E944C1680915404882359F094
:101CE000809154048150809354040E94AE048091EA
:101CF00054048823A9F70E948D2C882379F68091BB
:101D0000F804863039F781E00E94B314882311F378
:101D100080E00E9487148823E9F20E94AD170E9498
:101D20000D19E0E0F0EF19948C3009F449C08D30C2
:101D300038F4883069F18B3069F60E941926AECFED
:101D40008E3019F18E30F0F08F3021F60E94643120
:101D5000A5CF843059F0843030F0853009F0BACF07
:101D60000E943E389BCF0E942E2998CF0E94A61E2B
:101D700095CF0E94FD1292CF0E94FC448FCF0E940B
:101D800098428CCF0E94994B89CF0E94F61A86CF39
:101D90000E94AD170E944C1680915404882359F07C
:101DA000809154048150809354040E94AE04809129
:101DB00054048823A9F70E948D2C882359F36ECFF1
:101DC0000E9477116BCF0E94E02A68CF242F30E069
:101DD000C901880F991F820F931F880FE3CE7727C1
:101DE00067FD7095872F972F22EE34E040E050E09A
:101DF0000E94CD4C60537D4E8C4E9F4FBDCE8CE0EB
:101E00000E948714882309F427CF6E010894C11C0F
:101E1000D11CFF24B1E1AB2EB12CAC0EBD1EAFE046
:101E2000EA2E86010E941B01F801908381830E5FD8
:101E30001F4F0A151B05B1F7F60104C03196E017D4
:101E4000F10789F02081822F90E08F7090700D97BC
:101E500024F0822F8F708083282F2D3079F78E2FDA
:101E60008C198F3099F480E060E04F2D21E08601DD
:101E70000E943E3085E50E94C21A0E940D19F3941B
:101E8000F0E8FF1671F60E94AD17E6CEE082D6CFDD
:101E900010924404109287046091870470E061708E
:101EA000707062957295707F7627607F762782E0EA
:101EB00090E00E948B020E94C5301092D0041092D4
:101EC000BD0483E090E060E00E948B0284E090E03B
:101ED0006091BD040E948B0288E790E090939A0481
:101EE0008093990485E090E068E770E00E94950295
:101EF00080E1809300026091000287E090E00E9400
:101F00008B021092B70488E08093BA048091BA04DF
:101F10006091B70490E0019782959295907F982701
:101F2000807F9827682B8AE090E00E948B028DE0EA
:101F300090E060E00E948B02F89480ED92E1A3E1D2
:101F4000B0E08093090290930A02A0930B02B09331
:101F50000C0278948CE08093B40482E08093AD040A
:101F60008EE090E062E00E948B0210925B048FE0B2
:101F700090E060E00E948B0210E082E20E946A170B
:101F800083E20E946A170E940D1982E30E94CC0F1F
:101F90001F5F183291F777CF20EA3FE0E22FF32F4F
:101FA0003197F1F78A95D1F70895882309F41EC077
:101FB0009AEF20EA3FE0E22FF32F3197F1F79A955D
:101FC000D1F7E22FF32F3197F1F79A95D1F7E22F5E
:101FD000F32F3197F1F79A95D1F7E22FF32F31973D
:101FE000F1F79A95D1F7815009F0E5CF0895109255
:101FF000C6041092CF0408951F93CF93DF93EC0192
:10200000142F6F777885772309F44CC0462F50E062
:10201000888190E08F7790704817590779F121E017
:1020200030E00DC0D901FE01E20FF31F808190E086
:102030008F7790702F5F3F4F8417950709F127170F
:1020400088F3272F2F5F293030F128E0922F822F3D
:102050009150FE01E80FF11DDE01A90FB11D8C9119
:102060008083892F9923A1F71536C0F480E0862B51
:1020700088832887DF91CF911F910895A0E0B0E079
:10208000153670F480E0AC0FBD1F862B8C93DF916A
:10209000CF911F9108952223C9F6E6CF80E8E7CFBC
:1020A00080E8F1CF91E081E021E0D2CFCF93DF93C0
:1020B000EC0138853323B9F06F7770E0888190E0C8
:1020C0008F7790706817790789F0FE0120E008C0CB
:1020D000818190E08F77907031966817790739F099
:1020E0002F5F2317A8F3DF91CF91089520E03230BE
:1020F00068F0922F9F5FFE01E20FF11DDE01A90F34
:10210000B11D8C918083292F9317A0F3315038870C
:10211000DF91CF910895282F9091BD048091C00048
:1021200085FFFCCF90699093C6008091C00085FF29
:10213000FCCF822F8F778093C60027FD09C0909136
:1021400037028091C00085FFFCCF9093C6000895B0
:10215000909135028091C00085FFFCCF9093C6001E
:102160000895282F9091BD048091C00085FFFCCF79
:1021700090689093C6008091C00085FFFCCF822FAD
:102180008F778093C60027FD09C090913702809118
:10219000C00085FFFCCF9093C60008959091350252
:1021A0008091C00085FFFCCF9093C6000895982FC2
:1021B0008091C00085FFFCCF9093C60080E090E046
:1021C0000895909160048091610420E030E09817B8
:1021D00011F021E030E0C9010895909160048091F0
:1021E00061049817D1F3F89490916004E92FF0E01E
:1021F000EF52FB4F80819F5F909360049091600449
:102200009F7190936004789490E008959091600499
:1022100080916104981729F00E94ED10482F87FDE6
:1022200003C040E0842F0895582F52955F705F30AF
:10223000C9F3282F30E02F7030708091D00490E0E7
:102240002817390771F750935D04ECCF9091BD04C6
:102250008091C00085FFFCCF906B9093C600809169
:10226000C00085FFFCCF8BE78093C6008091C00043
:1022700085FFFCCF1092C6000895809144048230FF
:1022800049F08091C00085FFFCCF8CEF8093C600A1
:102290000E9426110895909146048913089580E0C4
:1022A0000E949E1E8FEF8093460408951F93182F5F
:1022B000962F6623B9F060E0809146048F3F09F0C5
:1022C00061E0953648F4812F895140E00E94871ED5
:1022D000109346041F910895812F895141E00E9477
:1022E000871EF6CF60E00E944B111F910895FF9268
:1022F0000F931F938091A80581708093A80580910A
:10230000A80580938F040E94AD178091A8058823AB
:1023100009F032C10E940D198BE090E00E94840206
:10232000809338028CE090E00E948402809339020E
:10233000FF2410E00E944C160E94F80C0E948D2C85
:10234000882309F04AC09091600480916104981735
:1023500069F00E94ED10682F87FD6DC080915D04CB
:10236000883009F4AEC0893009F479C0112371F4C2
:102370002091C604222349F48091CF04882329F4B4
:1023800080913607882309F4E2C010E087E10E94BB
:10239000DC14882379F28091A8058F5F8093A805CB
:1023A0008091A80581708093A8058091A8058093ED
:1023B0008F0480E00E9436178091A805882309F4D5
:1023C000B9CF80E00E94FE160E944C160E94F80CC5
:1023D0000E948D2C882309F4B6CF0E94261181E03B
:1023E00080934B06809129078093BC0510924C0680
:1023F0008091E806609129074091450620914B069F
:102400000FE816E00E94C92F60914506C8010E949E
:10241000022DFF2061F08BE090E0609138020E9475
:102420008B028CE090E0609139020E948B021F9138
:102430000F91FF900895482F42954F704F3009F447
:1024400098C0282F30E02F7030708091D00490E039
:102450002817390709F48DC010925D046BCF67FD12
:10246000BAC0062F0E94ED10482F112309F08ECF1D
:1024700050913802051748F0852F90E00F96202FD5
:1024800030E0821793070CF082C050913902051793
:1024900008F46ECF852F90E00C96202F30E0821745
:1024A00093070CF465CF051B87EC94E0602F0E9426
:1024B000FC0F8091C7048F778093D7062091C604C4
:1024C00059CF67FD84C0062F0E94ED10112371F5CE
:1024D00040913802041748F0842F90E00F96202F87
:1024E00030E0821793070CF06BC04091390204175B
:1024F00008F43ECF842F90E00C96202F30E0821716
:1025000093070CF435CF041B87EC94E0602F0E94F6
:1025100056108091CF04882309F42ACF8091C704F4
:102520008F778093D7062091C60424CF113009F409
:1025300056C089E10E943617009339028091A805A0
:1025400080938F042091C604FF24F39413CF84E07A
:102550000E94DC148823A1F485E00E94DC14882307
:1025600009F413CF10928F0489E10E94FE1612E045
:102570000DCF40935D04F2CE80E00E94FE16CACEDD
:1025800010928F0480E20E94FE1611E0FFCE051B20
:102590008EEB94E0602F0E94FC0F2091C6042093E4
:1025A0005E048091BE048F7780935F048091FD0468
:1025B00090915F048295807F890F80935F04DACECB
:1025C000041B8EEB94E0602F0E945610E6CF0E9411
:1025D000ED10082F79CF0E94ED10082F43CF80E235
:1025E0000E943617009338028091A80580938F04CB
:1025F0002091C604FF24F394BDCE1F930E94C217FE
:102600008091D0040E94D0170E944C1684E60E944C
:10261000CC0F0E944C1684E60E94CC0F0E944C16F0
:102620008FEF809346040E944C160E94F80C0E9483
:102630008D2C882311F59091600480916104981786
:1026400091F30E94ED10482F87FD1BC080915D041F
:10265000883049F1893039F747FD32C0142F0E9484
:10266000ED10682F812F0E9456110E944C160E9477
:10267000F80C0E948D2C8823F1F20E9426111F91E4
:102680000895582F52955F705F30B9F0282F30E0D1
:102690002F7030708091D00490E02817390769F0CE
:1026A00010925D04C0CF47FD0FC0142F0E94ED10A3
:1026B000682F812F0E944B11B6CF50935D04C6CF77
:1026C0000E94ED10182FCBCF0E94ED10182FEECFE7
:1026D0001F920F920FB60F920BB60F9211242F93E9
:1026E0003F934F935F936F937F938F939F93AF939A
:1026F000BF93EF93FF939091C6009A3F09F442C0B5
:102700009C3FA9F1983F09F44AC080916104E82FE9
:10271000F0E0EF52FB4F90838F5F809361048091D4
:1027200061048F71809361049091610480916004D1
:10273000981751F4809160048F5F809360048091BA
:1027400060048F7180936004FF91EF91BF91AF910E
:102750009F918F917F916F915F914F913F912F91B9
:102760000F900BBE0F900FBE0F901F901895809189
:102770008F04882349F380914404823029F70E9412
:102780002331E2CF809144048230F1F680918F04AE
:10279000882311F00E944D360E948900D5CF809188
:1027A0009404909195049093430480934204109272
:1027B00095041092940480914404823029F680910B
:1027C000630490916404892B31F05C9880915404E7
:1027D0008F5F8093540480915B04882371F0809113
:1027E0005B0490E00196909364048093630480916D
:1027F00054048F5F80935404A7CF8091420490913A
:102800004304969587959093640480936304EFCF77
:1028100080914404813009F05F98089599B1991F1F
:102820009927991F80916504882311F4992321F435
:102830009093650480E008959093650481E0089585
:1028400099B1991F9927991F80916604882311F0E7
:10285000992321F09093660480E008951092660415
:1028600081E008958AB1806F8AB98BB18F708BB97E
:1028700008958AB18F708AB98BB18F708BB9089522
:1028800080914404882321F45C9881E00E94CC0F5D
:102890005F9A0895AC01F8942898000000000000A9
:1028A0000000289A20E030E01EBC0DB407FEFDCFEA
:1028B0008EB5FA01E20FF31F80832F5F3F4F233065
:1028C000310591F77894089516980895169A089509
:1028D00020B1269526952F70822F90E02695322FD5
:1028E000369536952270322B880F991F282F247029
:1028F000322B880F991F880F991F8870382B8FE013
:10290000831B089580B1869586958F700895282F32
:10291000883188F4E82FE695E695E695F0E0E250F8
:10292000FB4F808190E0277002C0959587952A958E
:10293000E2F78170089580E00895282F883188F4A7
:10294000E82FE695E695E695F0E0EB50FB4F8081A9
:1029500090E0277002C0959587952A95E2F78170DF
:10296000089580E00895282F883188F4E82FE695AF
:10297000E695E695F0E0E750FB4F808190E0277008
:1029800002C0959587952A95E2F78170089580E0B9
:1029900008958091FE04882321F48091FF04882308
:1029A00019F090E0892F089590E080910005882328
:1029B000C9F791E0892F0895282F8831A0F4482F76
:1029C000469546954695277081E090E0382F01C0E6
:1029D000330F2A95EAF7A42FB0E0FD01EB50FB4F2F
:1029E0008081832319F420E0822F0895232F30E083
:1029F00020953095A250BB4F8C9190E0282339232D
:102A0000232B89F7342F3F5F832F63E00E94EC4C28
:102A1000E92FF0E0E250FB4F8081882321F720E08E
:102A2000832F8F5F0E94EC4CE92FF0E0E250FB4FC8
:102A300080818823C9F621E0D7CF1F93CF93DF93FE
:102A4000CCE4D2E010E088810E948714882329F426
:102A50001F5F21961D30B9F71FEF812FDF91CF91B6
:102A60001F9108951F93CF93DF93CCE4D2E010E041
:102A700088810E949D14882349F41F5F21961D3090
:102A8000B9F780E0DF91CF911F910895812F8F5F7B
:102A9000DF91CF911F9108951F93CF93DF93CCE4E3
:102AA000D2E010E088810E94B314882349F41F5FAC
:102AB00021961D30B9F780E0DF91CF911F910895E5
:102AC000812F8F5FDF91CF911F9108951F93CF9337
:102AD000DF93C4E4D2E010E088810E948714882349
:102AE00049F41F5F21961830B9F780E0DF91CF914C
:102AF0001F910895812F8F5FDF91CF911F910895CE
:102B00001F93CF93DF93C4E4D2E010E088810E944A
:102B10009D14882349F41F5F21961830B9F780E08F
:102B2000DF91CF911F910895812F8F5FDF91CF911A
:102B30001F9108951F93CF93DF93C4E4D2E010E078
:102B400088810E94B314882349F41F5F21961830AE
:102B5000B9F780E0DF91CF911F910895812F8F5FAA
:102B6000DF91CF911F910895CF93DF93C4E4D2E01A
:102B700088810E948714882349F4219682E0CC340E
:102B8000D807B1F780E0DF91CF91089581E0DF9120
:102B9000CF910895FF920F931F93CF93DF93C4E4D7
:102BA000D2E0FF2400E006C00F5F219682E0CC3423
:102BB000D80789F01881812F0E9487148823A1F7F4
:102BC000812F0E94B314882381F3F394219682E02D
:102BD000CC34D80779F781E0F81639F080E0DF913E
:102BE000CF911F910F91FF90089580E00730B9F7C2
:102BF00081E0F5CF1F93CF93DF93CAE3D2E010E0DB
:102C000088810E949D14882349F41F5F21961A3001
:102C1000B9F780E0DF91CF911F910895812F8F5FE9
:102C2000DF91CF911F9108958091680410926804FC
:102C3000089580E00895382F883100F5282F2770F7
:102C400081E090E0982F01C0990F2A95EAF7832F31
:102C5000869586958695A82FB0E0FD01EB50FB4F39
:102C60008081892369F4FD01E750FB4F808189232E
:102C700071F4A250BB4F8C91982339F480E00895F1
:102C8000832F0E94DC1982E0089583E00895832F4A
:102C90000E94E41981E00895EF92FF920F931F9331
:102CA000DF93CF9300D000D0CDB7DEB71092F504FC
:102CB0001092F9041092F6041092FA041092F7049C
:102CC0001092FB04809169048A3068F426960FB64E
:102CD000F894DEBF0FBECDBFCF91DF911F910F9152
:102CE000FF90EF9008951092690416987E01089461
:102CF000E11CF11CC7010E944A148091FE048C83E0
:102D00008091FF048D83809100058E8360E070E0E8
:102D100001E010E0E62FE695E695E695F0E0CB01C0
:102D200087709070980102C0220F331F8A95E2F7D6
:102D3000C901AF0142505B4FD701AE0FBF1F3C919D
:102D4000EF5FFA4F2081232B28238095FA013081F1
:102D50008323282B20836F5F7F4F68317105D1F665
:102D60000E946814982F96959093FD048093F30425
:102D7000169A40E050E0BE016C5F7F4FDA01AF5F12
:102D8000BA4FF701E40FF51F80818C93FB01E40F2C
:102D9000F51F2081FA01E250FB4F9081FA01EB50C0
:102DA000FB4F822F809589238083FA01E750FB4FE8
:102DB0009095922390834F5F5F4F43305105F1F61A
:102DC00090B1969596959F708091F104891721F0A6
:102DD00010926A049093F10480916A048F3630F067
:102DE0009093F2048091F2048093F10482E00E94B7
:102DF0008714809353040E940D1968CF282F8832BE
:102E0000C0F4E82FE695E695E695F0E0277081E0BE
:102E100090E001C0880F2A95EAF7DF01A559BB4F62
:102E20002C91282B2C93E059FB4F809520818223F5
:102E300080830895282F8832C0F4E82FE695E69520
:102E4000E695F0E0277081E090E001C0880F2A95B8
:102E5000EAF7DF01A059BB4F2C91282B2C93E559A1
:102E6000FB4F80952081822380830895282F88320C
:102E7000C8F4E82FE695E695E695F0E0277081E046
:102E800090E002C0880F991F2A95E2F78095DF0134
:102E9000A559BB4F2C9128232C93E059FB4F20813F
:102EA000822380830895282F883298F4E82FE695AE
:102EB000E695E695F0E0E059FB4F277081E090E061
:102EC00002C0880F991F2A95E2F7809520818223FE
:102ED00080830895282F883290F4E82FE695E695B0
:102EE000E695F0E0E559FB4F277081E090E002C0E5
:102EF000880F991F2A95E2F72081282720830895BB
:102F0000E82F883298F4282F277081E090E002C0E3
:102F1000880F991F2A95E2F7E695E695E695F0E089
:102F2000E059FB4F20812823822F089520E0822F33
:102F30000895982F969596959695EBE6F4E0E90F0F
:102F4000F11D208130E0877002C0359527958A9564
:102F5000E2F721703070C901089510926F04109249
:102F60006E0410926D0410926C0410926B04109217
:102F700074041092730410927204109271041092EF
:102F800070040895CF93DF93CAEBD2E089910E9439
:102F9000361782E0CA3CD807C9F7DF91CF91089570
:102FA000803108F00895E82FF0E0E654FD4F80816D
:102FB0000E94FE160895803108F00895E82FF0E091
:102FC000E654FD4F80810E94361708950F931F939A
:102FD000CF93DF93082FCAEBD2E010E007C08881BF
:102FE0000E94FE161F5F2196103149F01017B8F3AA
:102FF00088810E9436171F5F21961031B9F7DF9143
:10300000CF911F910F910895803108F00895E82F16
:10301000F0E0E654FD4F80810E941A170895803138
:1030200010F080E00895E82FF0E0E654FD4F808135
:103030000E9499170895803110F080E00895E82FDC
:10304000F0E0E654FD4F80810E948017089588319A
:1030500008F00895E82FF0E0EB56FD4F80810E94C4
:10306000FE160895883108F00895E82FF0E0EB5639
:10307000FD4F80810E941A170895883108F0089545
:10308000E82FF0E0EB56FD4F80810E94361708953F
:10309000CF93DF93C5E9D2E089910E94361782E091
:1030A000CD3AD807C9F7DF91CF910895E82F815025
:1030B000883008F00895F0E0E457FD4F80810E94C9
:1030C000FE1608950F931F93CF93DF93082FCDE83B
:1030D000D2E011E007C088810E9436171F5F219659
:1030E000193069F01017B9F7E12FF0E0E457FD4F00
:1030F00080810E94FE161F5F2196193099F7DF919B
:10310000CF911F910F910895E82F8150883008F0DA
:103110000895F0E0E457FD4F80810E94361708952E
:10312000E82F8150883008F00895F0E0E457FD4F13
:1031300080810E941A170895E82F8150883010F07E
:1031400080E00895F0E0E457FD4F80810E948017F1
:103150000895E82F8150883010F080E00895F0E065
:10316000E457FD4F80810E9499170895CF93DF9314
:10317000CDE8D2E089910E94361782E0C539D807A0
:10318000C9F7DF91CF9108958D3008F00895E82FA9
:10319000F0E0E355FD4F80810E94FE1608958D30CA
:1031A00008F00895E82FF0E0E355FD4F80810E947C
:1031B000361708958D3008F00895E82FF0E0E355B4
:1031C000FD4F80810E941A170895EDEAF2E0E80FA2
:1031D000F11D80810E9480170895CF93DF93CDEA7F
:1031E000D2E089910E94361782E0CA3BD807C9F71E
:1031F000DF91CF9108950E94ED1884E00E94361768
:1032000083E00E94361788E00E94361781E00E9412
:10321000361782E00E9436170895F894179820E038
:1032200030E090917504F901E059FB4F80819823BB
:10323000F901E559FB4F8081982B9EBD0DB407FE27
:10324000FDCF2F5F3F4F2530310559F7179A7894FE
:103250000895EBE6F4E0A0E7B4E080819D91892B2E
:10326000819384E0E037F807C1F70895EBE6F4E0D6
:10327000A0E7B4E09D91909580818923819384E0BB
:10328000E037F807B9F70895EBE6F4E0A0E7B4E01B
:1032900020819C91892F822319F09095922390830D
:1032A0001D92319684E0E037F80791F708951F9357
:1032B000182F84E00E943617123049F083E00E94F4
:1032C0003617113071F01F3F39F01F91089583E0D8
:1032D0000E941A171F91089584E00E94FE161F9104
:1032E000089583E00E94FE161F9108950F931F9387
:1032F000CF93DF93182F87FD50C086E10E943D18C1
:10330000812F829586958695837080FF29C085E1FF
:103310000E9427181F7349F11731A0F58FEF0E9403
:10332000571984E10E943D18012F10E0CBE0D0E056
:10333000C017D10731F0FE01EE55FD4F80810E948C
:1033400036172196C831D10599F70E551D4FF80152
:1033500080810E94FE16DF91CF911F910F910895F9
:1033600085E10E943D181F73B9F680E00E9457194D
:103370000E94ED1884E10E942718DF91CF911F91E0
:103380000F910895143268F0103370F4185181E0F1
:103390000E945719112329F6EBCF86E10E942718C6
:1033A000AFCF1C5080E0F4CF1C3318F4145282E0ED
:1033B000EFCF105383E0ECCFE5E9F2E0E80FF11D29
:1033C00080810E94FE160895E5E9F2E0E80FF11D04
:1033D00080810E9436170895EDE8F2E0E80FF11DB4
:1033E00080810E94FE160895EDE8F2E0E80FF11DDD
:1033F00080810E9436170895DF92EF92FF920F931B
:103400001F93CF93DF93F02EDE2C222371F1022F36
:10341000040FE42ECDE8D2E010E00BC0101758F4F2
:103420001F15D9F088810E94FE161F5F2196183063
:1034300049F01E1598F788810E9436171F5F219664
:103440001830B9F781E08D15A0F4DF91CF911F916D
:103450000F91FF90EF90DF900895E12FF0E0E35798
:10346000FD4F80810E941A17E0CF062F080FE82E2B
:10347000D1CFDD2071F088E00E94361781E00E94F4
:10348000FE16DF91CF911F910F91FF90EF90DF908B
:10349000089588E00E94FE1681E00E943617DF91B1
:1034A000CF911F910F91FF90EF90DF900895FF92C1
:1034B0000F931F93082FF62E84E00E94361783E0A7
:1034C0000E94361788E00E94361781E00E94361766
:1034D000102F04FD34C015FD29C007FD2CC016FDBA
:1034E00021C00E94ED18FF2099F0802F8F708D3041
:1034F00098F08BE10E94FE168CE10E94FE168FE090
:103500000E94FE168EE00E94FE168DE00E94FE16BE
:103510001F910F91FF9008950E94C4181F910F9161
:10352000FF90089581E00E94FE16DBCF83E00E94A9
:10353000FE1607FFD4CF88E00E94FE16D0CF84E0AD
:103540000E94FE16C8CFE9E5F2E0E80FF11D808188
:1035500008958C3008F00895E82FF0E0EF57FD4F04
:1035600080810E94FE160895CF93DF93C1E8D2E0D8
:1035700089910E94361782E0CD38D807C9F7DF91CC
:10358000CF91089590916B04982790936B0490913C
:103590006C04982790936C0490916D0498279093F5
:1035A0006D0490916E04982790936E0490916F042F
:1035B000982790936F040895AC0161157105A1F0EF
:1035C00020E0E0E0A0E0B0E0A40FB51F8C91E82778
:1035D000F0E0EE52FD4FE0812F5FA22FB0E0A61782
:1035E000B70790F38E2F0895E0E0FCCF0E944C16B1
:1035F0000E94F80C0E948D2C8823C1F30895EF924D
:10360000FF920F931F93CF93DF937C018B01611582
:10361000710561F0C0E0D0E0F701EC0FFD1F808183
:103620000E9409022196C017D107B0F3DF91CF9114
:103630001F910F91FF90EF90089522E420930405CD
:103640001092050522E020930605909307058093CC
:103650000805A4E0B5E0E0E08D91E827F0E0EE5247
:10366000FD4FE08185E0A930B807B1F7EC93CD01BB
:10367000059766E070E00E94FF1A089590E8909325
:1036800004051092050521E02093060580930705A7
:10369000A2EDB2E090915203FD01E90FF11D90817E
:1036A0009227FD01E90FF11D90819827A90FB11D07
:1036B0008C918093080584E095E065E070E00E94BD
:1036C000FF1A08951F920F920FB60F920BB60F922A
:1036D0001124DF92EF92FF920F931F932F933F934A
:1036E0004F935F936F937F938F939F93AF93BF930A
:1036F000CF93DF93EF93FF931091CE008091D1028F
:10370000882309F46EC08091780490917904895ED1
:10371000934008F080C080917604803408F089C01E
:10372000282F2F5FE82FF0E0EC5BFA4F10832093F7
:1037300076041092790410927804233008F451C072
:10374000709144059091450580E060914605462FB3
:1037500050E0482B592B30E0CA010496281739074E
:1037600008F43FC09A012D5F3F4FF901EC5BFA4F1F
:1037700010812115310509F401C190E0E0E0A0E0DD
:10378000B0E0AC5BBA4F8C91E827F0E0EE52FD4F11
:10379000E0819F5FA92FB0E0A217B30790F31E1737
:1037A00009F450C02115310509F4EAC090E0E0E0C9
:1037B000A0E0B0E0AC5BBA4F8C91E827F0E0EE52AD
:1037C000FD4FE0819F5FA92FB0E0A217B30790F3F0
:1037D0008E2F90E00E94E5011092760480E00E9416
:1037E0003E1BFF91EF91DF91CF91BF91AF919F91E0
:1037F0008F917F916F915F914F913F912F911F9189
:103800000F91FF90EF90DF900F900BBE0F900FBEC7
:103810000F901F9018950E94C2170E940D191093C7
:10382000440581E080937604109279041092780424
:10383000D8CF0E943E1B1092760410927904109209
:103840007804CFCF713809F48DC17238B0F5713179
:1038500009F426C1723108F096C0713051F170310F
:1038600031F080E00E943E1B10927604BACF6231A4
:10387000C1F780914705082F10E0000F111F000FBE
:10388000111F000F111F80914805080F111D02958F
:103890001295107F1027007F1027C9E4D5E0899189
:1038A000B8010E94691F0F5F1F4F85E0C935D80717
:1038B000B1F781E00E943E1BD7CF763809F430C1C2
:1038C000773808F073C0723809F47FC1753849F64B
:1038D0004330510509F0A5C030914705932F80E092
:1038E00020914805E22EFF24E82AF92AD0904905C4
:1038F000EAE3ED1508F4B6CF7093040510920505C0
:10390000F2E0DF0ED09206058EEFD80E3093070559
:1039100020930805DD2071F009E015E0E701CE01F4
:103920000E94AD1FF80181938F0121969E012E19EF
:103930002D15A8F380910605682F6D5F09F4E3C18A
:10394000A4E0B5E090E08E5F282F30E02B5F3A4F87
:103950008D919827E92FF0E0EE52FD4F9081A2174C
:10396000B307B1F7E62FF0E0EC5FFA4F90836F5F9B
:1039700084E095E070E00E94FF1A76CFE0E00FCF80
:1039800080E090E027CF703409F44EC1713409F023
:1039900068CF623009F065CF9091470580E02091B3
:1039A0004805820F911D0E94F1025ECF7738E9F140
:1039B000783809F056CF7093040510920505809170
:1039C0004705813009F465C1813008F056C180E1B6
:1039D00080930705109208058093090510920A0547
:1039E00084E047E0A7E0B0E068E070E0809306057F
:1039F00090E020E030E0F901EC5FFA4F80819827F9
:103A0000E92FF0E0EE52FD4F90812F5F3F4F2417DA
:103A100090F3AC5FBA4F9C9384E095E00E94FF1A4C
:103A200023CF80E00E943E1B1FCF80914705882353
:103A300009F001C14230510509F014CFE091480569
:103A4000E43008F00ECF89E180930405109205055B
:103A500080E1809306054E2F50E042955295507FAD
:103A60005427407F5427A7E0B5E008C0ED934F5F8F
:103A70005F4F35E0A731B30709F42EC1FA01E157D2
:103A8000F94FE0812E2F30E0C9018F7090700D97B3
:103A90006CF7207330702033310541F7EF7DE6CFAE
:103AA000623009F0DECE80914705082F10E0000F4C
:103AB000111F000F111F000F111F80914805080FE3
:103AC000111D02951295107F1027007F102789E1A4
:103AD000809304051092050580E180930605C7E0F8
:103AE000D5E0C8010E94AD1F89930F5F1F4F35E0DD
:103AF000C731D307B1F7DE015397E0E08D91E82796
:103B0000F0E0EE52FD4FE081CA17DB07B9F7E09312
:103B1000170584E095E064E170E00E94FF1AA4CEEE
:103B20009091470580E020914805E22EFF24E82A85
:103B3000F92A2EEFD22ED60E63506A3308F071CFD9
:103B4000DD2009F4B6CE09E415E0E701F801819122
:103B50008F01BE010E94691F21969E012E192D150D
:103B6000A8F3A7CE87E190E090930805809307051E
:103B700080ED90E090930A0580930905EAECF2E06D
:103B8000ABE0B5E081918D9322E0E03DF207D1F703
:103B900081E880930405109205058AE0809306056C
:103BA000A4E0B5E0E0E08D91E827F0E0EE52FD4FB3
:103BB000E08135E0A131B307B1F7EC93CD010D976A
:103BC0006EE070E00E94FF1A4FCE4230510509F0BE
:103BD00028CF30914705332309F468C090914805F8
:103BE00020E082E8809304051092050583E080932D
:103BF0000605309307059093080520930905A4E076
:103C0000B5E0E0E08D91E827F0E0EE52FD4FE08175
:103C100085E0AA30B807B1F7EC93CD01069767E0CD
:103C200070E00E94FF1A20CE8091990490919A042E
:103C30000E941D1B19CE813009F013CE423151056F
:103C400009F00FCEE0914805E43008F00ACE2E2F9F
:103C500030E0A9E4B5E022953295307F3227207F0D
:103C600032278D91F901E157F94F80832F5F3F4F44
:103C7000E5E0A935BE07A9F71CCE883009F0F1CDE3
:103C800081E08093070544E0A4E0B0E065E070E0E7
:103C9000ADCE88E08093070580E18093080582E03F
:103CA00045E0A5E0B0E066E070E0A0CE9091480568
:103CB000973860F4953870F4993139F1993120F0E2
:103CC000892F8158823030F020E08BCF9738C9F0AF
:103CD0009838D1F721E085CF5397E0E08D91E82720
:103CE000F0E0EE52FD4FE08185E0A731B807B1F773
:103CF000E0931705CD01439764E170E00E94FF1A3D
:103D0000B3CD24E06ECF90E02DCE20E16ACF2C9889
:103D1000803408F08FE3611160E4442349F090E0BF
:103D2000882349F0682B962B98B92C9A2D9A0895E0
:103D300090E88823B9F7962B98B90895882319F449
:103D40002D982C980895469A2C9808959F92AF929A
:103D5000BF92CF92DF92EF92FF920F931F93CF9378
:103D6000DF930E94C2178091BD040E94D0170E9469
:103D70004C160E941416BB249924AA24CC240E9419
:103D80004C160E94F80C0E948D2C882309F075C0F7
:103D90002B2D3CE02302C001112497E1D92ED80E2F
:103DA000EA2CE294EE0CEE0C80ECE822C0E0D0E0CD
:103DB00009C0802F0E94B314882319F52196CD30B5
:103DC000D10559F1FC2EFE01EE52FC4F0081802FEF
:103DD0000E949D14882369F31C2F1D0D812F6C2DCB
:103DE0004A2D0E94871E812F8E290E948B108C2FB6
:103DF0000E94C418CC24C394802F0E94B31488233B
:103E0000E9F28F2D8D0D8E290E94B1108F2D0E9409
:103E1000CF182196CD30D105A9F68FE00E949D14D0
:103E2000882309F444C081E08B150CF050C09B142A
:103E300029F08B2D0E9457190E940D1984E10E94D0
:103E40009D14882351F080E0AA2009F481E0A82E77
:103E50008823C9F188E00E94FE1686B190E08F7336
:103E60009070892BC1F49B2C0E944C160E94F80C78
:103E70000E948D2C882309F48BCF0E942611DF919C
:103E8000CF911F910F91FF90EF90DF90CF90BF9057
:103E9000AF909F9008950E94C914882321F380E079
:103EA0000E949E1E0E94ED18CC249B2CDDCF8EE03C
:103EB0000E949D14882309F4BACF2FEFB21609F49B
:103EC000B6CFBA94B4CF88E00E943617C6CFB39469
:103ED000AECF282FF89495E028980000000000004D
:103EE00000009EBD0DB407FEFDCF000000000000E5
:103EF00000001EBC0DB407FEFDCF8EB5289A000051
:103F000000000000000080FDE7CF289800000000BE
:103F100086E08EBD0DB407FEFDCF00000000289A9C
:103F2000000000000000000028980000000082E06F
:103F30008EBD0DB407FEFDCF7EBD0DB407FEFDCFD7
:103F40006EBD0DB407FEFDCF2EBD0DB407FEFDCF37
:103F500000000000289A78940895382FF89425E0FE
:103F6000289800000000000000002EBD0DB407FEE0
:103F7000FDCF00000000000000001EBC0DB407FED5
:103F8000FDCF8EB5289A000000000000000080FDE3
:103F9000E7CF28980000000083E08EBD0DB407FE37
:103FA000FDCF9EBD0DB407FEFDCF3EBD0DB407FE97
:103FB000FDCF000000001EBC0DB407FEFDCF8EB586
:103FC000289A78940895892F8F7184FD806E0895C2
:103FD000EF92FF920F931F93FA01D9018695808388
:103FE000862F90E08F709070959587959595879521
:103FF000959587958C93862F8770F80180836295BD
:104000006F70F70160831F910F91FF90EF900895FB
:10401000FC0130E022953295307F3227207F322715
:1040200020838081660F660F660F640F6F70862B8A
:104030008083089580917A04882349F087FD0EC01B
:1040400083E00E94FE1684E00E943617089583E004
:104050000E94361784E00E943617089583E00E947C
:10406000361784E00E94FE160895EF920F931F9377
:104070008091A4059091A50580E00E94DC1488231E
:1040800009F072C01091B905123009F486C0809110
:10409000B905843009F4A4C08091B90580FD3CC005
:1040A00080E00E94B314882321F41F910F91EF90B8
:1040B000089582E20E94FE168091B905823009F4CB
:1040C000BAC02091B3053091B4058091B905843010
:1040D00009F4AAC01092B9052115310591F0E091BB
:1040E000B605F0E0EE0FFF1FE152FC4F8081918199
:1040F0008217930730F0215030403093A50520936C
:10410000A40580914E04823009F4E7C010924E0459
:104110001F910F91EF9008950E94FA15482F882360
:1041200009F0BCC084E10E949D14882309F0A8C056
:1041300085E10E949D14882309F093C087E10E94C5
:104140009D14882309F082C083E00E949D14882377
:1041500009F4A6CF8091AF059091B0050E94260288
:1041600082E080934E049CCF81E08093B905109249
:10417000B4051092B30582E20E9436178091A4051F
:104180009091A50501960E94260282E080934E043C
:104190001091B905123009F07ACF0E94FA15482F14
:1041A000882309F474CF41502091B3053091B405B0
:1041B000C901880F991F880F991F880F991F220F17
:1041C000331F820F931F840F911D9093B40580932A
:1041D000B3058C599F4F0E94260210934E0457CF6F
:1041E0000E94FA15482F882309F456CF4150209198
:1041F000B3053091B405C901880F991F880F991F25
:10420000880F991F220F331F820F931F840F911D58
:104210009093B4058093B30588539F4F0E94260264
:1042200082E080934E0438CF28533F4F3093B4053B
:104230002093B3054FCF2091B3053091B4052C598D
:104240003F4F3093B4052093B3053FCF8091B7051E
:104250009091B80501960E94260282E080934E0458
:1042600073CF84E08093B9051092B4051092B30522
:1042700088EC90E00E94260282E080934E045ECF9C
:1042800012E01093B9051092B4051092B30584E6BC
:1042900090E00E94260210934E044ACF83E0809360
:1042A000B90541502091B3053091B405C901880F7B
:1042B000991F880F991F880F991F220F331F820F94
:1042C000931F840F911D9093B4058093B3050E94B2
:1042D000260282E080934E0425CF0E94B41A80917A
:1042E000450660914B064091BE0520914C06009119
:1042F0004506E090BC050E94FC1908CF962F80313E
:1043000010F08FEF0895682F70E0660F771F6F5FD2
:10431000734F892F0E94691F80E008959B018031AF
:1043200020F5682F70E0FB01EE0FFF1FE152FC4FFC
:104330008081918128173907A0F0009749F08150BA
:10434000660F771F6050744F0E94691F80E00895C8
:1043500080E0660F771F6050744F0E94691F80E0F5
:104360000895C901009759F7F3CF8FEF0895803171
:1043700098F470E06050784F90E00024969587950F
:104380000794969587950794982F802D680F791F2D
:104390008CE06030780710F08FEF0895842F0E9432
:1043A000691F80E00895EF92FF920F931F93CF93C0
:1043B000DF93C82FD0E0CC0FDD1FCC0FDD1FCC0F5B
:1043C000DD1FC60FD11DC05CDF4FCC0FDD1FC295B6
:1043D000D295D07FDC27C07FDC27EE24FF24870125
:1043E000000F111F0C571A4FF80180819181892FFE
:1043F000BE010E94691FF801808191812196BE0152
:104400000E94691F0894E11CF11C2196F0E1EF164F
:10441000F10429F7DF91CF911F910F91FF90EF9059
:10442000089590E0880F991F8F5F934F0E94AD1FF2
:1044300090E008950F931F93082F10E0000F111FB5
:10444000C8018050944F0E94AD1F90E00196015228
:104450001C4FF801208131818217930708F49C01D9
:10446000C9011F910F9108958091F3048093B605BF
:104470008091B6050E941A229093B0058093AF05F3
:104480008091B6050E9411229093B8058093B705DC
:104490002091B7053091B8058091AF059091B00596
:1044A0002817390720F01092B8051092B7058091AF
:1044B000A4059091A505E091B605F0E0EE0FFF1F71
:1044C000E152FC4F608171810E94F84C9093A505E8
:1044D0008093A4050895803198F470E06050784F7F
:1044E00090E0002496958795079496958795079474
:1044F000982F802D680F791F8CE06030780710F0BE
:104500008FEF0895CB010E94AD1F0895CF92DF92E7
:10451000EF92FF920F931F93DF93CF930F92CDB73C
:10452000DEB7C090A405D090A5050894C11CD11C8D
:1045300080E00E94DC14882309F0C0C01982109129
:10454000B905123009F4CDC08091B905843009F461
:1045500048C18091B90580FD18C080E00E94B31465
:10456000882329F08091B905882309F000C1E981E9
:10457000E13009F42FC10F90CF91DF911F910F917E
:10458000FF90EF90DF90CF9008950E94FA15282FAA
:10459000882309F0D0C084E10E949D14882309F08B
:1045A00062C185E10E949D14882309F04DC187E115
:1045B0000E949D14882349F0C090B705D090B8059B
:1045C0000894C11CD11CF1E0F98383E00E949D1482
:1045D000882309F0A9C089E00E949D14882309F06E
:1045E00096C189E00E94B314882309F04AC18AE089
:1045F0000E949D14882309F018C18AE00E94B31418
:10460000882309F4AACF8CE10E943617E091B60501
:104610002091AF053091B005F0E0EE0FFF1FE152A1
:10462000FC4F808191812817390708F096CF80913F
:10463000AF059091B00501969093B0058093AF05BA
:104640008091B6056091AF057091B0050E948E21F2
:104650008091B6050E941A229093B0058093AF0511
:104660006091AF057091B005615070408091A405D4
:104670009091A50586179707E8F47B010894E10857
:10468000F10801C079018091B6051E2D6E2D0E94A2
:104690006B22482F8091B6051F5F612F0E94B721C2
:1046A0009701215030408091A4059091A5058E1569
:1046B0009F0540F388E0809384044FCF81E080938E
:1046C000B9051092B4051092B3058093810482E27B
:1046D0000E94361781E089831091B905123009F0E4
:1046E00033CF0E94FA15482F882309F42DCF41506B
:1046F0002091B3053091B405C901880F991F880F27
:10470000991F880F991F220F331F820F931F840F49
:10471000911D9093B4058093B3058C599F4F0E94CF
:10472000260210934E0410CFC090AF05D090B00574
:1047300081E0898350CF83E08093B9052150809137
:10474000B3059091B4056C01CC0CDD1CCC0CDD1CC8
:10475000CC0CDD1C880F991FC80ED91EC20ED11CAF
:10476000D092B405C092B305E1E0E98314CF82E2B0
:104770000E94FE16109281048091B905823009F4DE
:10478000E6C02091B3053091B4058091B90584301D
:1047900009F4D6C01092B90581E0809384042115F4
:1047A000310569F0E091B605F0E0EE0FFF1FE15230
:1047B000FC4F808191818217930708F0B7C08091E8
:1047C0004E04823009F4CEC010924E04E981E130EB
:1047D00009F0D1CEC6010E94260282E080934E04E9
:1047E000CACE0E94FA15482F882309F4B2CE415050
:1047F0002091B3053091B405C901880F991F880F26
:10480000991F880F991F220F331F820F931F840F48
:10481000911D9093B4058093B30588539F4F0E94D8
:10482000260282E080934E0494CE8CE10E94FE1614
:104830001092B4051092B305C090A405D090A505C0
:104840000894C11CD11CD9CE84E08093B905109284
:10485000B4051092B30588EC90E00E94260282E035
:1048600080934E04A4CE12E01093B9051092B405C3
:104870001092B30584E690E00E94260210934E0445
:1048800090CE8BE10E943617E090A405F090A5052C
:104890000894E11CF11C8091AF059091B005E816D9
:1048A000F90608F0A4CE8091B6051E2D6E2D0E944B
:1048B0006B22482F8091B6051150612F0E94B721BD
:1048C0000894E11CF11C8091AF059091B005E816A9
:1048D000F90648F38091AF059091B0050197909348
:1048E000B0058093AF058091B6056091AF057091DA
:1048F000B0050E948E218091B6050E941A229093E5
:10490000B0058093AF0588E08093840470CE8BE17E
:104910000E94FE161092B4051092B305C090A40533
:10492000D090A5050894C11CD11C5BCE215030400D
:104930003093A5052093A40587E0809384043FCF9E
:1049400028533F4F3093B4052093B30523CF2091D4
:10495000B3053091B4052C593F4F3093B4052093E3
:10496000B30513CF0E94B41A8091450660914B069F
:104970004091BE0520914C0600914506E090BC0593
:104980000E94FC1921CFEF92FF920F931F93809109
:10499000F3048093B6058091B6050E941A22909385
:1049A000B0058093AF058091B6050E9411229093C7
:1049B000B8058093B7052091B7053091B80580916F
:1049C000AF059091B0052817390720F01092B8056F
:1049D0001092B7058091A4059091A505E091B605C8
:1049E000F0E0EE0FFF1FE152FC4F608171810E94E9
:1049F000F84C9093A5058093A4058091B60560912D
:104A0000A4057091A5050E946B228093AC0580914E
:104A1000B6056091AC0544E056E02CEB35E00EEBBA
:104A200015E0F0EDEF2EF6E0FF2E0E94E81F81E08A
:104A300080934C068091D0068D3010F01092D006F5
:104A40000E94BE2C8091D0068093D7061F910F91B3
:104A5000FF90EF900895AF92BF92CF92DF92EF92C6
:104A6000FF920F931F93CF93DF93C82EDD24CC0CBE
:104A7000DD1CCC0CDD1CCC0CDD1CC60ED11C80E476
:104A800090E0C80ED91ECC0CDD1CC294D29410EF5D
:104A9000D122DC24C122DC24AA24BB24C6010E942A
:104AA000AD1FD82FC0E07501EE0CFF1CE4E8F5E067
:104AB000EE0EFF1EF701D183C08300811181C60174
:104AC00001960E94AD1F90E0082B192BF70111836E
:104AD00000830894A11CB11C82E090E0C80ED91E8E
:104AE00090E1A916B104D1F6DF91CF911F910F91FA
:104AF000FF90EF90DF90CF90BF90AF90089510920D
:104B0000AE0584E20E9436170E94AD170E94441938
:104B100010924A0680E00E949E1E08951092AD05F4
:104B200010924A061092A60580E00E949E1E0E94E6
:104B3000AD170E9444190E94141608958091AA0589
:104B40009091AB05682F6770969587959695879598
:104B5000969587958F700E948D306091AA0570910F
:104B6000AB059B0140E050E0DA01C901807090780C
:104B7000A070B070892F9A2FAB2FBB2780938B0426
:104B8000DA01C90180709074A070B070892F9A2FDB
:104B9000AB2FBB2780938904207030724070507017
:104BA000232F342F452F552720938A041092BF05B9
:104BB000872F8F7184FD806E089581E08093AD050D
:104BC00081E20E94FE1610928904809189048093EC
:104BD0008A0480918A0480938B041092A605109217
:104BE0004A0680918405909185059093AB0580934A
:104BF000AA058F5F9F4F89F01092B2051092BF05F2
:104C0000109297040E949E2580937A048091450417
:104C100080FDFCCF81E08093A6050E94C217089515
:104C200081E08093AE0584E20E94FE160E94C217C6
:104C30000895BF92CF92DF92EF92FF920F931F934E
:104C400080913607882309F405C384E00E94422D31
:104C50001092A9058091A9058093A8051092B90525
:104C60001092B5051092B4051092B3050E94C324AA
:104C70008091E806609129074091450620914B06F6
:104C80000FE816E00E94C92F8091450660914B06FF
:104C90004091BE0520914C060091C205E090BC05F4
:104CA0000E94FC19CC2467E0B62E0E944C160E948C
:104CB000F80C1091CF06133099F01430A0F5113094
:104CC00009F459C00E94602F882379F70E942F2F82
:104CD0000E944C160E94F80C1091CF06133069F711
:104CE0000E94482D882309F066C10E94BA2E8823AD
:104CF00021F01092810410928F040E943215D82E58
:104D0000882301F3DA940E94ED188D2D0E94C418B7
:104D1000D092D006809136078823A1F68091D006E4
:104D20008093D706CFCF143061F01D3059F681E063
:104D30000E94A2368091CF068D3021F210928F040E
:104D4000C1CF0E94482D882309F01BC1CC2009F453
:104D50005AC081E0C81609F46DC288E00E94B314FD
:104D60008823E1F11092810410928F0484E00E9464
:104D7000422DCC24A7CF0E94482D882309F07DC165
:104D80000E94862283E00E94DC14882309F02AC155
:104D900083E00E94B314882309F020C19091B605E6
:104DA0008091F304981711F00E94C3248091CF06DC
:104DB000813011F010928F0480913607882309F01A
:104DC00009C10E948D2C882309F47CCF1F910F917B
:104DD000FF90EF90DF90CF90BF9008950E94321522
:104DE000D82E882381F0DA940E94ED188D2D0E9430
:104DF000C418D092D00680913607882321F4809180
:104E0000D0068093D7068091B905882371F4CC2011
:104E100009F4E6C18091B60586958093FD04DD20F6
:104E200009F07DC180E00E94A236CC2011F40E94DE
:104E3000862283E00E94DC14882309F047C187E1C1
:104E40000E94DC14882309F04DC186E10E94DC1425
:104E5000882309F453C180914C06882309F05CC172
:104E60008091D0068093D706E090A405F090A50528
:104E70008091A905882309F058C180914B068823A9
:104E800009F44AC010E0209129073091450680912D
:104E9000D70690E082959295907F9827807F9827FB
:104EA0008093AC058091AC05220F220F220F230FB7
:104EB000210F2F70282B2093AC058091B6056091AF
:104EC000A4057091A5054091AC050E94B7211F5F14
:104ED0008091A4059091A50501969093A5058093D6
:104EE000A4050894E11CF11C8091A4059091A505EE
:104EF000E091B605F0E0EE0FFF1FE152FC4F60813C
:104F000071810E94F84C9093A5058093A40580912F
:104F10004B06181708F4B7CF8091A805882309F02D
:104F200017C1B092840480918404873009F423C1AE
:104F300080918404883009F457C1809184048130C1
:104F400009F4B4C08091CF06843011F010928F0420
:104F500080913607882309F4B5C080918E04813092
:104F600009F0B0CE10928E040E948D2C882309F493
:104F7000A9CE1F910F91FF90EF90DF90CF90BF903F
:104F800008950E94AD1782E20E94FE1681E0809390
:104F90008F0481E20E94FE168091450660914B06C7
:104FA0004091BE0520914C0600914506E090BC055D
:104FB0000E94FC19CBCE0E94AD1711E01093810422
:104FC00084E20E94FE168091D0060E94C4181093BD
:104FD0008F048BCE84E00E94422DF3CE83E20E94A8
:104FE0003617DCCE1092A5051092A4058091B60567
:104FF0006091A4057091A5050E946B228093AC0579
:105000008091B6056091AC0544E056E02CEB35E0AC
:105010000EEB15E0A0EDEA2EA6E0FA2E0E94E81FA6
:1050200081E080934C068091D0068D3010F0109274
:10503000D0068091D0068093D7060E94BE2C809126
:10504000E806609129074091450620914B060FE83C
:1050500016E00E94C92F8091450660914B06409151
:10506000BE0520914C060091C205E090BC050E944F
:10507000FC1983E20E94FE168BCE0E94AD1782E2DD
:105080000E94FE1610938F0481E20E9436178091D1
:10509000450660914B064091BE0520914C0600915B
:1050A0004506E090BC050E94FC196ACE109284046B
:1050B000CC2009F447CF0E94ED188091D0060E94C1
:1050C000C41840CF81E00E94422D47CF81E08093F9
:1050D000A80583E20E941A1787E10E94DC14882346
:1050E00009F4B3CE81E08093A90580E00E941A17ED
:1050F00086E10E94DC14882309F0ADCE86E10E948F
:105100009D14882309F40FCFCC2009F40CCF809193
:105110004C06882309F4A4CE0E94BE2CA1CE81E0C7
:105120000E94382DCC24C39484CE1092A90580917E
:10513000B6056E2D0E947E218091B6050E94112237
:105140009093B8058093B70580E00E94361795CEFE
:105150001092A8058091B605B7010E948E2180911A
:10516000B6050E941A229093B0058093AF0583E2A2
:105170000E943617D6CE8091B6056091A405709135
:10518000A5050E946B228093AC058091B6056091C5
:10519000AC0544E056E02CEB35E00EEB15E090ED6D
:1051A000E92E96E0F92E0E94E81F81E080934C06DC
:1051B0008091D0068D3010F01092D0068091450677
:1051C00060914B064091BE0520914C060091C205AE
:1051D000E090BC050E94FC1981E080938404ADCE70
:1051E0000E944D2FD82E16CE8091B6056091A40551
:1051F0007091A5050E946B228093AC058091B60545
:105200006091AC0544E056E02CEB35E00EEB15E088
:10521000B0EDEB2EB6E0FB2E0E94E81F81E08093FC
:105220004C068091D0068D3010F01092D00610926E
:10523000840483CE0E94AD17C092810484E20E9450
:10524000FE168091D0060E94C418C0928F0452E0CE
:10525000C52E83CD81E00E94422DFACCEF92FF92C1
:105260000F931F9380913607882309F4A5C184E02A
:105270000E94422D1092A9058091A9058093A8054E
:105280001092B9051092B5051092B4051092B305AD
:105290000E94C3248091E806609129074091450649
:1052A00020914B060FE816E00E94C92F8091450619
:1052B00060914B064091BE0520914C060091C205BD
:1052C000E090BC050E94FC1908C0143009F457C0D6
:1052D0000E94602F882309F490C00E944C160E94FF
:1052E000F80C1091CF06113081F70E94482D8823C9
:1052F00009F08AC083E00E94DC14882309F0A5C06D
:1053000083E00E94B314882309F0EFC00E94352087
:105310009091B6058091F3049817E1F00E94C324A0
:105320008091E806609129074091450620914B063F
:105330000FE816E00E94C92F8091450660914B0648
:105340004091BE0520914C060091C205E090BC053D
:105350000E94FC198091CF06813011F010928F04C9
:1053600080913607882309F04BC00E948D2C88233A
:1053700009F4AECF1F910F91FF90EF9008950E9416
:10538000482D882309F0E0C086E10E94DC148823C0
:1053900009F0CEC083E00E94DC14882309F0BCC071
:1053A00088E00E94DC14882309F0A7C088E00E94EE
:1053B000B314882329F08091B505882309F0E1C052
:1053C0000E9435208091CF06843011F010928F0416
:1053D00080913607882309F48CC080918E04813037
:1053E00009F076CF10928E040E948D2C882311F63E
:1053F0000E94602F882309F070CF0E942F2F6DCF5D
:1054000084E00E94422DB1CF0E94AD1782E20E943B
:10541000FE1610938F0481E20E9436178091450694
:1054200060914B064091BE0520914C0600914506C7
:10543000E090BC050E94FC1981E00E94620283E0BA
:105440000E94DC14882309F45BCF1092A50510920A
:10545000A4058091B6056091A4057091A5050E94F0
:105460006B228093AC058091B6056091AC0544E059
:1054700056E02CEB35E00EEB15E070EDE72E76E014
:10548000F72E0E94E81F81E080934C068091D006A1
:105490008D3010F01092D0068091D0068093D70600
:1054A0000E94BE2C8091E806609129074091450634
:1054B00020914B060FE816E00E94C92F8091450607
:1054C00060914B064091BE0520914C060091C205AB
:1054D000E090BC050E94FC1983E20E94FE1683E066
:1054E0000E94B314882309F411CF83E20E94361777
:1054F0000DCF81E00E94422D70CF81E08093B505F1
:10550000809381040E94AD1784E20E94FE16809170
:10551000D7060E94C4184ACF81E08093A80583E291
:105520000E94FE161092A90580E00E94361738CF1F
:1055300081E08093A90580E00E94FE161092A805E4
:1055400083E20E94361726CF0E94AD1782E20E94A6
:10555000FE1681E080938F0481E20E94FE16809106
:10556000450660914B064091BE0520914C06009186
:105570004506E090BC050E94FC1981E00E94620291
:1055800003CF1092B505109281040E94ED1884E2B9
:105590000E94361782E20E94FE16809145066091B5
:1055A0004B064091BE0520914C0600914506E090C7
:1055B000BC050E94FC1904CF81E00E94422D5ACE06
:1055C000EF92FF920F931F9310927C048091360705
:1055D000882309F49EC184E00E94422D1092A905FF
:1055E0008091A9058093A8051092B9051092B50580
:1055F0001092B4051092B3050E943422E2E0FE2E10
:1056000007C0113009F494C00E94602F8823D9F09C
:105610000E944C160E94F80C1091CF061330E9F04E
:10562000143078F31430E9F11D3071F781E00E94F5
:10563000A2368091CF068D3039F310928F040E94EC
:10564000602F882329F70E942F2F0E944C160E945A
:10565000F80C1091CF06133019F70E94482D8823BB
:1056600009F0E8C00E94BA2E882321F0109281042C
:1056700010928F040E943215882331F2182F115096
:105680000E94ED18812F0E94C4181093D0068091BB
:105690003607882309F0B8CF8091D0068093D706CB
:1056A000B3CF0E94482D882309F0EDC08091B90541
:1056B000882309F4DBC083E00E94DC14882329F0EE
:1056C00080917C04813009F40DC187E10E94DC14D3
:1056D000882309F0C4C080E00E94DC14882309F00C
:1056E000A0C080E00E94B314882309F08DC080918F
:1056F000CF06843011F010928F04809136078823F2
:1057000009F4A7C080918E04813009F07DCF1092FA
:105710008E0480917C04882309F076CF0E948D2C22
:10572000882309F471CF1F910F91FF90EF90089596
:105730000E94482D8823B1F58091B905882309F48A
:1057400056C083E00E94DC14882379F081E08093C6
:105750007C0480917C04882309F4B8C083E20E9411
:10576000FE161092A5051092A4050E943520909176
:10577000B6058091F304981711F00E9434228091AD
:10578000CF06813011F010928F0480913607882364
:1057900029F284E00E94422D0E948D2C882309F476
:1057A00033CFC1CF0E94AD1782E20E94FE16109344
:1057B0008F0481E20E9436178091450660914B0666
:1057C0004091BE0520914C0600914506E090BC0535
:1057D0000E94FC1980917C04882309F47BC083E239
:1057E0000E94FE168091B905882309F0AACF0E9475
:1057F0004D2F9091B60596959093FD04882309F05E
:10580000A0CF0E94A2369DCF82E20E94FE16109287
:10581000B90580914E04823009F46AC010924E049A
:1058200066CF81E08093B90582E20E943617F0923C
:105830004E0457CF0E94AD1711E01093810484E20B
:105840000E94FE168091D0060E94C41810938F0407
:1058500009CF81E00E94422D10927C0453CF81E059
:105860008093A90580E00E941A1735CF0E944D2F22
:105870009091B60596959093FD04882309F01BCF6F
:105880000E94A23618CF0E94AD1782E20E94FE1637
:1058900081E080938F0481E20E94FE16809145068C
:1058A00060914B064091BE0520914C060091450643
:1058B000E090BC050E94FC1980917C04882371F063
:1058C00083E20E941A170E940D19F0CE83E20E9413
:1058D000361747CF83E20E9436172ECF83E20E940D
:1058E0003617F1CF8093A80583E20E94FE16EDCE15
:1058F0000E94B41A8091450660914B064091BE0506
:1059000020914C0600914506E090BC050E94FC19D0
:1059100085CF81E00E94422D61CE9091F20480916A
:10592000F804891731F08091F2048093F80481E043
:10593000089580E0089580914C06882391F080912D
:1059400004068093E8068091BC0580932907809126
:10595000BE058093450680914C0680934B061092BD
:105960004C0680914B06882329F080914B0680934A
:105970004B06089581E080934B06089580910406BC
:105980008093E8068091BC05809329078091BE052D
:105990008093450680914C0680934B0610924C06EE
:1059A0000895833059F0843050F0843029F080918C
:1059B000D0068093D70608951092D00608958230BD
:1059C000B0F70895FC0187858F708D30C1F030E00D
:1059D00020E190E080818F708E3061F09F5F319682
:1059E0009217C0F3892F913118F48150832B0895B9
:1059F00080E1FBCF9923B1F780E0832B089530E15C
:105A00002FE0E7CF1F93DF93CF930F92CDB7DEB791
:105A1000162F0E94E22C898389818F708F5F80937B
:105A200000041093C205898184FD08C08CE0809336
:105A3000FF030F90CF91DF911F91089580E1809334
:105A4000FF030F90CF91DF911F910895E82FF0E0B1
:105A5000EF73F070EE5FFB4F808108954093C005B7
:105A6000609303068093CF0681E0809348060895F3
:105A7000882339F0809103068093CF0681E08093DC
:105A8000480608958093CF0681E0809348060895E4
:105A900080914806882319F01092480681E0089505
:105AA0003F924F925F926F927F928F929F92AF92AE
:105AB000BF92CF92DF92EF92FF920F931F93CF93FB
:105AC000DF93462E4A015901662309F4C4C09C01A4
:105AD000E90100E0FF241FEFDD2466247724B2E013
:105AE0005B2E33243394CE010E94E22CF301ED525D
:105AF000F94F8083C0802FE0C222C39440E050E081
:105B000012C01E251F7BF1F4F501E00FF11D30825C
:105B1000FF2009F070C0DD24D3940F5F4F5F5F4F0B
:105B20001E2D4C1588F5642FFE01E40FF51FE08053
:105B30002E2D30E0C9018F7090700F9709F455C079
:105B4000DD20F9F6F501E00FF11D5082EF2DF0E0B8
:105B5000D401AE0FBF1FEC926295607FE35BF94FFB
:105B60006083F3940024220F331F001C220F331F85
:105B7000001C232F302DDD24D394D2220F5F4F5FE2
:105B80005F4F1E2D4C1578F20894611C711C6096B5
:105B9000641408F4A8CF003408F061C08F2DF5011B
:105BA000E00FF11D10820F5F0034C8F39FE39F15D3
:105BB00050F09FEFEF2DF0E0E35BF94F9083F3940B
:105BC0002FE32F15B8F7DF91CF911F910F91FF9021
:105BD000EF90DF90CF90BF90AF909F908F907F908D
:105BE0006F905F904F903F900895F501E00FF11D89
:105BF0001082DD2492CFEF2DF0E03197E80DF91DF2
:105C0000E082FA94EF2DF0E0F394E35BF94FA0818A
:105C1000AF70BA2FBF5F808182958F70682F70E060
:105C2000CB018B0F911D40970CF0BA2F0024220F4F
:105C3000331F001C220F331F001C232F302DDD24A7
:105C4000D394D22262957295707F7627607F7627F3
:105C5000B62BB08362CF00E0FF2480E0A0CF8F2D71
:105C6000A5CF2F923F924F925F926F927F928F9229
:105C70009F92AF92BF92CF92DF92EF92FF920F93DB
:105C80001F93CF93DF935C01562E3A01790166236F
:105C900009F45DC0482EEC0130E060E0DD24DA94C8
:105CA000CC2480E000E010E05FE04EE0342E2DE0F8
:105CB000222E93ED892E96E0992E800E911EF401EE
:105CC00070817F707F5FDE0190E0442D41950BC0B5
:105CD0005C93223089F0C42ECA0E3F5F9F5F1196FD
:105CE000822F9717D0F4F701E30FF11D20812130A7
:105CF00079F7882349F45C93F301E60FF11DD08016
:105D00006F5FDC9222E0E7CF5C93F501EC0DF11DB3
:105D1000808180648083DC92DECF903158F4FE0174
:105D2000E90FF11D30829F5F05C0FE01E90FF11DF3
:105D300050839F5F9031C8F3F401808184FD2F86EA
:105D40000F5F1F4F6096822F051508F4B2CFDF91C9
:105D5000CF911F910F91FF90EF90DF90CF90BF9068
:105D6000AF909F908F907F906F905F904F903F90FB
:105D70002F9008958091C0050E94B314882339F0B4
:105D8000809103068093CF0681E0809348060895B2
:105D90001092AE0584E20E94361710927E0480E0D5
:105DA0000E9436170E9444190E9448180E94C21788
:105DB0008091FC040E94D01780E00E949E1E0895EE
:105DC00081E08093AE0584E20E94FE160E94C21715
:105DD00080E00E94D01780E00E949E1E08951092DD
:105DE0004A060E9448180E94C2170E9444198091D6
:105DF000FC040E94D0171092460681E20E943617DA
:105E000080E00E949E1E109236078CEF0E94D710F1
:105E100008951092BF0581E08093460681E20E94BA
:105E2000FE1680E00E949E1E80914404882321F487
:105E30008091450480FDFCCF1092450410926204CD
:105E40001092A3048091A3048093A50481E0809321
:105E50004A06809336078AEF0E94D71008958091F2
:105E60008F04882311F480E0089581E00E94DC14FF
:105E7000882321F081E080939004089581E00E94BE
:105E80009D14882381F380E00E948714882359F3AE
:105E900082E08093900481E0089588E00E94871456
:105EA000882369F09091CF0688E08093C005909395
:105EB000030683E08093CF0681E08093480608952F
:105EC00080914404823011F080E008950E94061110
:105ED00080932B0780E00895AF92BF92CF92DF921C
:105EE000EF92FF920F931F93CF93DF935B01C82E26
:105EF000DD24C294D29450EFD522DC24C522DC24C8
:105F0000EE24C0E0D0E0FF24F39405C02196F39482
:105F1000F1E1FF16B1F085010C0F1D1FC6018C0FBA
:105F20009D1F0E94AD1FF8018083EE2079F78081CC
:105F30008F708E3059F7EF2C2196F394F1E1FF1614
:105F400051F7EE20A1F490E1F50187858F708D3037
:105F5000B9F0892F81508F70DF91CF911F910F91F0
:105F6000FF90EF90DF90CF90BF90AF9008959E2D5F
:105F7000915051F791E0F50187858F708D3049F789
:105F8000903110F08EE1E8CF892F81508F708061C1
:105F9000E3CFBF92CF92DF92EF92FF920F931F93C6
:105FA000CF93DF936801E82EFF24EE0CFF1CE60E72
:105FB000F11CEE0CFF1CEE0CFF1CEE0CFF1CE40EA3
:105FC000F11CE294F29470EFF722FE24E722FE2403
:105FD00030E022953295307F3227207F3227B22E53
:105FE000222379F0C0E0D0E086010C0F1D1FC7010D
:105FF0008C0F9D1F0E94AD1FF80180832196CB1549
:1060000098F3DF91CF911F910F91FF90EF90DF9068
:10601000CF90BF900895EF92FF920F931F93CF936D
:10602000DF93182F062F0E940D19E12EFF24EE0C8E
:10603000FF1CEE0CFF1CEE0CFF1CE00EF11CE294AA
:10604000F294A0EFFA22FE24EA22FE24C0E0D0E07F
:10605000FE01E852F94F8081BE016E0D7F1D0E9446
:10606000691F2196C031D10599F70E940D19DF9162
:10607000CF911F910F91FF90EF900895CF92DF92F3
:10608000EF92FF920F931F93CF93DF93E22E68015D
:10609000082F10E0000F111F060F111D000F111F18
:1060A000000F111F000F111F040F111D02951295F3
:1060B000107F1027007F1027FF24E294F29480EFD6
:1060C000F822FE24E822FE24FE2C82E00E94FE1626
:1060D0000E940D19EE2099F0C0E0D0E0F601EC0F1F
:1060E000FD1F8081B8016C0F7D1F0E94691F82E037
:1060F0000E94CC0F0E94F80C2196CF1578F382E015
:106100000E9436170E940D19DF91CF911F910F91B8
:10611000FF90EF90DF90CF900895EF92FF920F9352
:106120001F93CF93DF93182F062F0E940D19E12E96
:10613000FF24EE0CFF1CEE0CFF1CEE0CFF1CE00E0F
:10614000F11CE294F29440EFF422FE24E422FE24B7
:10615000C0E0D0E0CE018E0D9F1D0E94AD1FFE015C
:10616000E852F94F80832196C031D10599F71092FA
:106170007E0480E00E9453170E940D19DF91CF9199
:106180001F910F91FF90EF90089580914404882310
:1061900049F40E94C80080914404813049F00E9473
:1061A000321408950E94C900809144048130B9F7E7
:1061B0000E94391408950F931F938091D006809305
:1061C000D70680914C068823C9F0809104068093FD
:1061D000E8068091BC05809329078091BE058093D5
:1061E000450680914C0680934B0610924C06809198
:1061F0008104823088F01F910F91089590912907B2
:106200008091BC059817B9F380918104823098F78A
:106210008091BC05809329078091E8066091290749
:106220004091450620914B060FE816E00E94C92FC9
:10623000609145068091D1069091D2060E94022D70
:106240001F910F9108951092360780E00E949E1EC4
:106250008CEF0E94D71080914404813011F00E948D
:10626000081410928D061092A3048091A3048093C9
:10627000A5041092BD058FE896E09093D206809316
:10628000D1068091F8048D3031F0833021F08B30CD
:1062900011F0873011F40E94DB3080915204882382
:1062A00061F480915104882309F408958091510488
:1062B0000E94B110109251040895809152040E94DE
:1062C000B11010925204EDCF4F925F926F927F9275
:1062D0008F929F92AF92BF92CF92DF92EF92FF92F6
:1062E0000F931F93CF93DF9381E08093CF0680932A
:1062F000480610E0C0E0D0E0BB24FF24F394AA24B9
:10630000AA9442E0E42E34E0932E23E0822E90E221
:10631000792E80E1682E0FE0502EB1E14B2E0E94C5
:106320004C160E94F80C8091CF06873009F4DFC02C
:10633000883008F07EC0843009F489C2863009F4C0
:1063400048C2813061F780914806882331F010926D
:1063500048060E94AD170E940D1987E10E94DC14C7
:10636000882361F08091CF0697E19093C0058093D8
:10637000030687E08093CF06F092480688E00E94EB
:10638000DC14882361F08091CF0698E09093C005DB
:106390008093030686E08093CF06F092480681E062
:1063A0000E94DC14882351F08091CF06F092C00542
:1063B000809303069092CF06F09248068EE00E94EA
:1063C000DC14882359F09091CF068EE08093C005AD
:1063D000909303065092CF06F092480682E00E9406
:1063E000DC14882351F08091CF06E092C0058093A1
:1063F00003066092CF06F09248069091F2048091D5
:10640000F804891709F48BCF8091F2048093F80483
:10641000DF91CF911F910F91FF90EF90DF90CF9080
:10642000BF90AF909F908F907F906F905F904F90B4
:106430000895803109F449C1813109F4D9C08F3000
:1064400009F06DCF80914806882349F010924806E4
:10645000F09284048091F3048093830410E080918F
:10646000C0050E94B314882349F0809103068093ED
:10647000CF06F0924806112309F01CC30E94801534
:10648000882369F0982F9150933048F48091B70495
:10649000981729F09093B704F092840411E080914A
:1064A000B704813009F4A5C280918404882309F4DB
:1064B00036CF109284040E94B6180E94C2178091B1
:1064C000B7048F5F0E9456188091B704813009F09D
:1064D00026CF8091BA0481500E94D0170E944C169A
:1064E0000E94F80C8091CF06873009F021CF80916F
:1064F0004806882361F010924806F092840480E0F8
:106500000E94FE168091F3048093830410E0809132
:10651000C0050E94B314882349F08091030680933C
:10652000CF06F0924806112309F097C20E94801509
:10653000882379F0982F9150933058F48091440437
:10654000981739F0909344040E94C530F092840467
:1065500011E083E00E949D14882369F080918704F4
:106560008F5F809387048091870481708093870474
:10657000F092840411E09091F304809183049817C1
:1065800079F08091F30480938304809183048530B3
:1065900038F48091830480935B04F092840411E0CA
:1065A00086E10E949D14882309F0B3C18091840480
:1065B000882309F4B4CE109284040E94B618809106
:1065C00044048F5F0E94561883E20E943617809120
:1065D0008704882309F4BFC20E94C2178091440433
:1065E000823009F06FC080915B040E94D0176AC0AE
:1065F000809148068823C1F010924806F0928404E6
:10660000A09282048091AD04813009F485C2823069
:1066100009F47FC2843009F479C2883009F473C266
:1066200082E00E94FE1610E08091C0050E94B31423
:10663000882349F0809103068093CF06F0924806A4
:10664000112309F056C20E948015882341F1982F2A
:106650009150943020F580918204981701F1909325
:106660008204F092840480918204882309F077C226
:1066700041E080918204823009F477C280918204E3
:10668000833009F478C2242F30E0C901880F991FA4
:10669000820F931F880F8093B4044093AD048091C0
:1066A0008404882309F43BCE109284040E94B61817
:1066B00080918204843008F032C2809182048F5F1E
:1066C0000E9456180E940D192ACE809148068823F0
:1066D00059F010924806F092840410920104F0924E
:1066E000820410E0C0E0D0E08091C0050E94B314A5
:1066F0008823B1F0809103068093CF06F09248067C
:10670000112351F080918204813009F47AC2809182
:106710008204823009F442C210924E04F0920104C5
:1067200080E00E949D14882361F080918204823071
:1067300041F0E092820482E20E941A17F0928404EF
:1067400010E00E94FA15282F882389F0CE01880FC7
:10675000991F880F991F880F991FCC0FDD1FC80F35
:10676000D91F2150C20FD11DE092840411E0009185
:106770008204023009F459C180918404882309F409
:10678000CECD80918204813009F484C1809182044D
:10679000823009F0C4CD80918404823009F0EEC1CA
:1067A0000C2F8BE10E9436178CE10E9436170023D4
:1067B00039F0B7FC6EC21B141CF48CE10E94FE166B
:1067C000802F90E00E942602F0924E0410928404E2
:1067D000A6CD80914806882339F010924806109281
:1067E00084041092820410E08091C0050E94B314CA
:1067F000882349F0809103068093CF06F0924806E3
:10680000112309F069C180918204882309F4D9C059
:1068100020918204213009F4B7C0209182042230F3
:1068200009F486C080918404813009F4A2C080916B
:106830008404823009F073CD109284040E94C21740
:106840008091BD040E94D0170E940D1968CD8091DF
:106850004806882339F010924806F092840410927A
:10686000820410E08091C0050E94B314882331F1A6
:10687000809103068093CF06F09248061123E1F041
:1068800080918204882311F4F09282048091820422
:10689000813210F070928204909100028091820403
:1068A000981751F080918204809300026091000259
:1068B00087E090E00E948B0210924E040E94FA152D
:1068C000382F882389F0809182042AE0829FC001BA
:1068D000112480938204809182048150830F8093DD
:1068E0008204E092840411E080918404882309F4F6
:1068F00016CD9091000280918404823009F41CC16D
:10690000892F90E00E942602F0924E041092840497
:1069100006CD9091030687E18093C005909303060E
:106920004092CF06F092480680E00E9436173ECE95
:106930009091F30480918304981759F08091F304A7
:106940008093830420938404809183048093BD0406
:1069500011E089E00E94B314882309F463CF1092F8
:1069600082048BE10E94361780918404813009F003
:106970005ECF109284040E94C2178091D0040E94BE
:10698000D0170E940D19CBCC9091F3048091830411
:10699000981759F08091F304809383042093840422
:1069A000809183048093D00411E08AE00E94B314A4
:1069B000882309F432CF109282048CE10E943617AA
:1069C0002CCF8AE00E949D14882309F0B8C089E08A
:1069D0000E949D14882309F41BCF8BE10E94FE16B0
:1069E000E0928204E09284048091F3048093830413
:1069F0000FCF909183048091F304981709F454CD3C
:106A00008091F30480938304909183049F5F92307C
:106A100008F424C18091BA04981709F445CD9093E5
:106A2000BA04F092840411E03FCD89E00E949D14E5
:106A3000882331F01B1424F400938404BB24BA94FB
:106A40008AE00E949D14882309F496CEB7FE94CE66
:106A5000E0928404BB24B3948FCE8091870490E0AD
:106A60008170907082959295907F9827807F98276B
:106A7000609144046F70682B82E090E00E948B026A
:106A800060915B048FE090E00E948B0280E00E94A6
:106A900036174CCD80918404823009F4E1C0809196
:106AA000990490919A040E942602F0924E0410924A
:106AB00084046CCE8091BA046091B70490E0019791
:106AC00082959295907F9827807F9827682B8AE0FF
:106AD00090E00E948B02D2CC83E090E06091D004E1
:106AE0000E948B0284E090E06091BD040E948B02C2
:106AF0008ACE8EE090E06091AD040E948B0282E02D
:106B00000E943617A0CD809282048ACDE092820442
:106B100087CDF092820484CD1092820481CD85E0ED
:106B20000E94561886E00E94561887E00E94561868
:106B300088E00E945618C6CD90918204E1CE8CE187
:106B40000E94FE16F0928204F09284048091F30475
:106B5000809383043CCF83E20E94FE163DCD42E049
:106B600080918204823009F089CD44E080918204D2
:106B7000833009F088CD48E080E38DCD8DE090E052
:106B80000E948402282F992787FD909597FD7DC04C
:106B9000082F27FD77C0BB24B39403CEB7FC70C089
:106BA00081E0C536D10508F062C0992787FD909530
:106BB0008C9F60018D9FD00C9C9FD00C1124BC2C0D
:106BC0006C2D772767FD7095872F972F22EE34E085
:106BD00040E050E00E94CD4C60537D4E8C4E9F4F64
:106BE0000C2DF8946093090270930A0280930B02B3
:106BF00090930C028DE090E0602F0E948B027894BD
:106C00008BCDC431D10580F181E0CD32D80710F0B1
:106C1000CCE2D1E0F8948091990490919A048C1779
:106C20009D07D1F0D0939A04C09399048091990460
:106C300090919A040E94F1028091990490919A0493
:106C40009093B3048093B2046091990470919A0474
:106C500085E090E00E949502789459CD92E0DACEDA
:106C6000CE010E94260221CFC4E1D0E0D3CFC0E004
:106C7000D0E0BB2460ED72E183E190E000E0B1CFB1
:106C80008FEF8FCFBB24BA948CCD909581959F4F79
:106C90007FCF8BE10E94FE168ECD0F931F93DF9363
:106CA000CF930F92CDB7DEB705B180E00E949E1E54
:106CB00010928D0610924504109262041092910475
:106CC00010925A041092A3048091A3048093A50407
:106CD0001092BD058FE896E09093D2068093D1067E
:106CE000109145060E94E22C898389818F708F5F05
:106CF000809300041093C205898184FD21C08CE03B
:106D00008093FF0383E080933607809144048130B1
:106D100011F00E9440148AEF0E94D71083E0809304
:106D20004C04109251041092520405FF03C081E0FC
:106D30000E94CC0F0F90CF91DF911F910F9108957A
:106D400080E1DECFEF920F931F93982F882309F4F1
:106D500095C0813029F080E01F910F91EF90089548
:106D600080914806882309F0F9C00E948015882385
:106D700099F1982F915080914C06882341F480918D
:106D800045068093BE058091E806809304068091B5
:106D9000BE05891770F48091BE05981B9F5F909384
:106DA0004C0680914C06853008F446C184E08093FF
:106DB0004C0680913607882309F441C1809145062D
:106DC00060914B064091BE0520914C060091C20592
:106DD000E090BC050E94FC1984E10E949D14882368
:106DE00009F0DEC085E10E949D14882309F0CEC021
:106DF00080913607882321F5909129078091BC0561
:106E00009817F1F08091BC05809329078091E806DE
:106E1000609129074091450620914B060FE816E046
:106E20000E94C92F8091450660914B064091BE0596
:106E300020914C060091C205E090BC050E94FC190F
:106E400080913607882329F480914C06882309F025
:106E5000D4C00E949A15982F882309F47CCF809182
:106E600082049150981709F076CF809103068093A1
:106E7000CF0681E08093480680E06ECF0E948015A7
:106E8000982F8823D1F584E10E949D14882309F46A
:106E90009FC01092BC0588E00E94FE1681E00E940F
:106EA000361780913607882309F055CF909129072E
:106EB0008091BC05981709F44ECF8091BC05809352
:106EC00029078091E80660912907409145062091A5
:106ED0004B060FE816E00E94C92F8091450660918D
:106EE0004B064091BE0520914C060091C205E090F2
:106EF000BC050E94FC1980E02FCF8091FD04809397
:106F0000040601E000934C06192F11501093BE05A2
:106F100084E10E948714882309F44BC01092BC05B9
:106F200088E00E94FE1681E00E94361710938204CA
:106F30008091CF06809303068DE08093CF0681E099
:106F4000809348061092D00680913607882309F472
:106F50004FC081E01F910F91EF9008951092480665
:106F600090938F048091450660914B064091BE0539
:106F700020914C060091C205E090BC050E94FC19CE
:106F80000E948015882309F427CFF3CE81E08093F7
:106F9000BC0588E00E94361781E00E94FE1628CFCB
:106FA0001092BC0588E00E94FE1681E00E94361710
:106FB00019CF85E10E948714882309F4B7CF009385
:106FC000BC0588E00E94361781E00E94FE16AECF15
:106FD00085E10E949D14882309F463CF81E08093AA
:106FE000BC0588E00E94361781E00E94FE1659CF4A
:106FF00082E00E94D12C81E0ADCF80910406809385
:10700000E8068091BC05809329078091BE05809396
:10701000450680914C0680934B0610924C06809159
:10702000E806609129074091450620914B060FE83C
:1070300016E00E94C92F0DCF80914C06B8CE8091EA
:1070400004068093E8068091BC058093290780910F
:10705000BE058093450680914C0680934B061092A6
:107060004C068091E80660912907409145062091E1
:107070004B060FE816E00E94C92FA0CE2F923F9238
:107080004F925F926F927F928F929F92AF92BF9238
:10709000CF92DF92EF92FF920F931F93DF93CF93E4
:1070A0000F92CDB7DEB70E944C161092D006809199
:1070B000D0068093D70680913607882311F40C946C
:1070C000174284E08093CF0681E0809348066624CF
:1070D000992488245524772473945CE0452E43E05A
:1070E000342E34E0232E0E944C160E94F80C10918E
:1070F000CF061830E9F0193008F04EC0153009F409
:10710000A5C4163008F096C0113009F42FC214300F
:1071100009F413C40E94602F882329F70E942F2F9F
:107120000E944C160E94F80C1091CF06183019F7E7
:1071300080914806882349F0109248060E94AD17B6
:1071400083E20E94FE16709281048091C0050E9425
:10715000B3148823A1F0809103068093CF06709228
:107160004806109281048091E806609129074091B9
:10717000450620914B060FE816E00E94C92F0E9499
:107180008015882309F013C50E949A15882311F2EF
:1071900081500E94F419BECF1B3009F4E1C21C30AB
:1071A000C0F5193009F481C21A3009F0B3CF8091CB
:1071B00048068823F1F01092480680E00E94FE16EF
:1071C0000E940D198091E8066091290740914506BB
:1071D00020914B060FE816E00E943E3080E00E94AE
:1071E00036170E940D192092CF0670924806109211
:1071F000810480918404882331F02092CF0670921C
:10720000480610928404809184048F5F80938404E4
:1072100081CF1C3009F47AC11D3009F07BCF81E0A9
:107220000E94A2368091CF068D3009F473CF109260
:107230008F0470CF163009F4F9C0173009F06ACF07
:1072400080914806882389F1109248060E94AD1764
:1072500060914B068FE896E049EE56E023EC35E06E
:107260000E94502D80E00E94FE161092840489E056
:10727000809382041092830480914B06882391F0BE
:1072800020E0E22FF0E0ED52F94F908180918304ED
:107290008F5F9F70890F809383042F5F80914B06CF
:1072A000281778F366249924552480E00E94DC1482
:1072B000882311F06624639488E00E94DC148823FC
:1072C00011F082E0682E87E10E94DC14882311F01F
:1072D00003E0602E80918204893009F424C78091F4
:1072E0008204813009F4F8C680918204882309F46D
:1072F0002CC580918204882329F080918204807FAC
:1073000009F45CC0109182048EE00E949D148823D1
:1073100051F080918204806180938204F5E0F093C3
:107320008404B2E05B2E8FE00E949D14882351F00C
:107330008091820480628093820485E0809384043B
:107340005524539484E10E949D14882349F0809130
:10735000820480648093820495E090938404552491
:107360008EE00E94B314882339F080918204807EDD
:1073700080938204209284048FE00E94B3148823B7
:1073800039F080918204807D80938204209284046D
:1073900084E10E94B314882339F080918204807BB9
:1073A000809382042092840480918404853009F4BF
:1073B0008BC580918404843009F476C58091820461
:1073C000883009F469C48091840490E083709070DF
:1073D000892B09F079C4662009F49CCE60914B0694
:1073E0008FE896E049EE56E023EC35E00E94312E1E
:1073F0008091E806609129074091450620914B064F
:107400000FE816E00E943E3081E0681609F46FC56F
:1074100092E0691609F474C0F3E06F1609F07ACEB1
:1074200087E08093CF067092480674CE809148061C
:107430008823D9F0109248060E94AD1760914B0640
:107440008FE896E049EE56E023EC35E00E94502D9F
:1074500084E20E94FE161092840410928304F3E6E4
:10746000F093820466249924882480E00E94DC142E
:10747000882311F06624639488E00E94DC1488233A
:1074800011F022E0622E80918204833609F419C63D
:1074900080918204813009F4B5C5809182048330E3
:1074A00009F43DC580918204882309F48FC480913A
:1074B000840490E083709070892B09F057C4662093
:1074C00009F428CE60914B068FE896E049EE56E02D
:1074D00023EC35E00E94312E8091E8066091290767
:1074E0004091450620914B060FE816E00E943E3081
:1074F00081E0681609F4FBC492E0691609F00ACE2F
:10750000E6E0E093CF067092480604CE80914806EC
:10751000882389F01092480690917F0480914B0651
:10752000981709F4B3C6709284048091030680937F
:10753000CF06709248068091C0050E94B31488233C
:1075400009F4E8CD809103068093CF067092480637
:1075500080918404882309F429C68DE00E9436179F
:1075600082E00E9436170E940D19D4CD8091480602
:107570008823E9F01092480680E00E9462020E948F
:10758000AD1782E20E94FE1610938F0481E20E94E2
:1075900036178091450660914B064091BE052091BB
:1075A0004C0600914506E090BC050E94FC1980E065
:1075B0000E94A23680E00E949D14882329F085E075
:1075C0008093CF067092480683E00E949D14882322
:1075D00059F08091CF063092C0058093030688E071
:1075E0008093CF067092480688E00E94DC148823BE
:1075F00029F096E09093CF067092480687E10E94AA
:10760000DC14882329F0E7E0E093CF067092480667
:107610008BE00E94DC14882359F09091CF068BE018
:107620008093C005909303068093CF06709248061E
:107630008DE00E94DC14882359F09091CF068DE0F4
:107640008093C005909303064092CF06709248063F
:107650008091CF06813011F010928F04809136070F
:10766000882321F02092CF06709248069091F20470
:107670008091F804891709F44DCD8091F20480932C
:10768000F8040F90CF91DF911F910F91FF90EF9031
:10769000DF90CF90BF90AF909F908F907F906F9032
:1076A0005F904F903F902F900895809148068823D7
:1076B00081F01092480682E20E94361781E00E9413
:1076C0009E1E80E00E949E1E81E00E9462027092D7
:1076D0008F0480913607882309F4C1C290918204F7
:1076E0008091C1059817C9F0909082048091C105DE
:1076F0008093820480918404833009F4E4C58091EE
:107700008404823050F08091BB05882331F4E091ED
:107710008204F0E0ED53FA4F708286E10E949D14DE
:10772000882329F08091BB05882309F407C580913F
:107730008404833009F4E0C386E10E94B3148823F3
:1077400009F4E8CC80918404823009F0E3CC709293
:10775000840480E00E949E1E82E00E943617DACCEC
:1077600080914806882361F01092480682E20E94C8
:1077700036178FE00E94FE160E940D1910928404A5
:107780008091C0050E94B314882309F442C08091FF
:1077900003068093CF067092480680918404882364
:1077A00091F58091E806309129072091450690E0F7
:1077B000880F991F830F911D880F991F880F991F9C
:1077C000880F991F280F2093800480914B06809387
:1077D0007F048823C1F090E0A0E0B0E0282F30E0E3
:1077E00022953295307F3227207F3227FD01E157E5
:1077F000F94F8081AB5FB94F8C939F5FA92FB0E0A9
:10780000A217B3079CF38FE00E9436178DE00E9409
:1078100036178DE00E949D14882309F47BCC80915B
:107820008404882309F076CC80917F04882309F4AE
:1078300071CC709284048091E80620912907109100
:10784000450690E0880F991F820F911D880F991FA0
:10785000880F991F880F991F180F8091800418179F
:1078600009F458CC8DE00E94FE1682E00E94FE16BC
:107870000E940D199091800480914B06882309F491
:1078800042C0A92EBB24A294B294B0EFBB22BA246A
:10789000AB22BA247501C12EDD24C294D294A0EF8C
:1078A000DA22DC24CA22DC2400E010E0C7010E94B6
:1078B000AD1F882E0157194FF8018083C6010E9421
:1078C000AD1FB7010E94691F882DB6010E94691F74
:1078D00082E00E94CC0F0E94F80C0894E11CF11C7D
:1078E0000894C11CD11C8E2D8A19082F10E080919C
:1078F0004B0690E082959295907F9827807F9827FD
:10790000081719079CF2109145068FE896E00E942F
:10791000E22C898389818F708F5F8093000410939C
:10792000C205898184FD8DC58CE08093FF0382E0D0
:107930000E9436170E940D19EDCB809148068823CE
:10794000E9F0109248060E94AD1782E20E94FE16EE
:1079500070928F0481E20E94FE168091450660912C
:107960004B064091BE0520914C0600914506E090E3
:10797000BC050E94FC1981E00E94620283E00E9423
:10798000DC14882309F445C080914C06882309F053
:107990006AC4909129078091BC05981781F0809165
:1079A000BC05809329078091E806609129074091E2
:1079B000450620914B060FE816E00E94C92F609102
:1079C0004B068FE896E049EE56E023EC35E00E9446
:1079D000502D80E090E0FC01ED53FA4F10820196AB
:1079E00080349105C1F782E08093810410922C07C6
:1079F0001092830410928204109284041092BB05AA
:107A00007092860489E08093CF067092480699248C
:107A10009A948091CF06843011F010928F04809157
:107A20003607882321F47092CF0670924806809121
:107A30008E04813009F06ECB10928E049091F20486
:107A40008091F804891709F018CE64CB809148061C
:107A50008823C9F0109248060E94AD1770928404E2
:107A60008FE896E00E94E22C282F2F702F5F209342
:107A7000820490E0929582958F7089279F70892764
:107A80008170809383048EE00E941B16823009F47B
:107A9000D9C08AE00E941B16823009F4B9C089E07F
:107AA0000E941B16823009F4C1C08FE00E949D1411
:107AB000882391F03092840480918304882311F408
:107AC00040928204809183048F5F8093830480912D
:107AD00083048170809383048091840480FF21C09B
:107AE000809184048150809384048091830488234E
:107AF00009F4CEC180918204803108F4DEC381E0B4
:107B00008093820483E00E94FE1680918204882381
:107B100009F0BBC181E080938204809182040E94BD
:107B2000E61780E00E94B314882309F4F3CA809119
:107B300084048230B8F182E0809381048FE896E07B
:107B400061E049EE56E023EC35E00E94502D909123
:107B5000820480918304811180E191509F70892B70
:107B60008093D3068FE896E061E049EE56E023EC7F
:107B700035E00E94312E8091E806609129074091FE
:107B8000450621E00FE816E00E943E308091E806AD
:107B9000609129074091450620914B060E94C92F0C
:107BA000109281047092CF0670924806B3CA182FC3
:107BB0001150812F0E94EC198091E80690912907BD
:107BC000E82EFF24EE0CFF1CE90EF11CEE0CFF1C4E
:107BD000EE0CFF1CEE0CFF1CE10EF11CE294F29483
:107BE00070EFF722FE24E722FE248701005F1F4F7B
:107BF0008FE0B7010E94691F82E00E94CC0F0E94B3
:107C0000F80C0894E11CF11CE016F10689F7BCCAD7
:107C1000809182048F708F5F8093820430928404FD
:107C200089E00E941B16823009F03FCF80918204C8
:107C300090E00E968F7090708F5F809382043092E8
:107C4000840433CF80918404823008F4B8C38091D7
:107C500082048F5F80938204309284041ACF81E083
:107C60000E949E1E80E00E949E1E1092860410922A
:107C7000A5047092CF0670924806109281048091FC
:107C8000E806609129074091450620914B060FE8D0
:107C900016E00E94C92F22CDE92DF0E0ED53FA4FF6
:107CA0005082939480918304981610F06624639414
:107CB00070928404109282048091840490E0837016
:107CC0009070892B09F487CB0E94C21780914B06D4
:107CD0008823B1F090E080E001C08E2FE92FF0E022
:107CE000ED52F94FE081EF70EF5FE80F981618F052
:107CF0009E1608F4F1C29F5F80914B06981768F3B7
:107D000084E00E94361783E00E94361788E00E94C4
:107D100036178091840480FD13C0E2E05E1609F4FA
:107D200092C3F1E05F1609F492C3552031F084E06C
:107D30000E94FE1683E00E94FE1688E00E94FE1656
:107D40000E940D191092840446CB86E10E94DC1437
:107D5000882309F4CECAE92DF0E0ED53FA4F5080A4
:107D60007092820482E080938404C3CA0E94C21786
:107D7000E92DF0E0E35BF94F80818F3FD1F0108176
:107D800012951F7000810F70010F0F5F101738F0F0
:107D900010C0812F0E9404181F5F101750F48091AB
:107DA000840480FDF6CF812F0E94D0171F5F10172B
:107DB000B0F38091840480FFF4C1882D60E00E94BC
:107DC000571A109284040E940D1979CB86E10E9403
:107DD0009D14882309F08AC20E943215882309F075
:107DE000BCC287E10E94B314882329F0FFE39F0EF1
:107DF0009F22709284048EE00E949D14882321F0BB
:107E000080E1882A709284048FE00E949D14882368
:107E100021F090E2892A7092840484E10E949D14EA
:107E2000882321F0E0E88E2A7092840485E10E9484
:107E30009D14882321F0F0E48F2A709284048EE050
:107E40000E94B314882321F08FEE8822709284045C
:107E50008FE00E94B314882321F09FED8922709255
:107E6000840484E10E94B314882321F0EFE78E227A
:107E70007092840485E10E94B314882309F417CB1F
:107E8000FFEB8F227092840412CB8091820443CE48
:107E900080918204813108F413C281E080938204CE
:107EA00083E00E94361731CE112359F0809182046D
:107EB000882339F4939480918304981610F06624F3
:107EC0006394709284047ACA112309F0EDC1809101
:107ED0008204882309F4E8C1662029F4E92DF0E042
:107EE000ED53FA4F508282E08093840462CA60921C
:107EF000CF06609248060EC90E94CA15882309F46D
:107F00001BCC82E08093840486E10E94871488233E
:107F100009F012CC709284040E949E1E0DCC0E9427
:107F20003215182F0E944C15882319F4112309F4D7
:107F3000B9CAE92DF0E0E751F94F808280E00E9454
:107F40009E1E82E00E94CC0F9394FFE3F91518F473
:107F500010928304992470928404109282048FE01A
:107F600088228EE00E948714882311F090E1892AEC
:107F70008FE00E948714882311F0E0E28E2A84E1CA
:107F80000E948714882311F0F0E88F2A85E10E946F
:107F90008714882311F080E4882A112309F482CA07
:107FA000812E8A949FE089228EE00E948714882384
:107FB00011F0E0E18E2A8FE00E948714882311F0EF
:107FC000F0E28F2A84E10E948714882311F080E870
:107FD000882A85E10E948714882311F090E4892A79
:107FE000E82DF0E0EF73F070EE5FFB4F482D407826
:107FF000808160E00E94871E82E08093840430923A
:10800000820450CA86E10E94B314882309F0DCC1BF
:108010008EE00E949D14882349F0882D8095807100
:108020009FEE8922882A82E0809384048FE00E9458
:108030009D14882349F0882D80958072EFED8E2263
:10804000882A82E08093840484E10E949D1488231E
:1080500049F0882D80958078FFE78F22882A82E07A
:108060008093840485E10E949D14882349F0882D23
:10807000809580749FEB8922882A82E08093840413
:108080000E943215182F882309F407CA80E00E9445
:108090009E1E82E00E94CC0F11501F70E0EF8E22D6
:1080A000812AE82DF0E0EF73F070EE5FFB4F482D72
:1080B0004078808160E00E94871E82E08093840483
:1080C000ECC988E00E94B314882309F4E1C9109236
:1080D000820470928404DCC986E10E94B314882370
:1080E00019F088E0809382048EE00E949D1488231A
:1080F00029F082E08093840412E0512E8FE00E94E8
:108100009D14882329F082E080938404552453949D
:1081100084E10E949D14882309F4E6C882E08093DC
:1081200084045524E1C887E10E94B314882309F42C
:10813000D6C81092820470928404D1C882E08093E1
:1081400084040E94B415882311F030928404E091D5
:108150008204F0E0ED53FA4F82E08083E0918304E3
:10816000F0E0E751F94F808080924906E82DF0E079
:10817000EF73F070EE5FFB4F482D4078808160E038
:108180000E94871E80918204981639F09090820494
:10819000809183048F5F8093830482E00E94FE16A7
:1081A000C6CA882D61E00E94571A0BCE82E00E9459
:1081B000FE160E940D199091E80620912907309132
:1081C000450680917F048823C9F1E92EFF24EE0C37
:1081D000FF1CE20EF11CEE0CFF1CEE0CFF1CEE0C63
:1081E000FF1CE30EF11CE294F29460EFF622FE24F1
:1081F000E622FE248701A0E0B0E0FD01EB5FF94F2D
:108200008081A157B94F8C93B8010E94691F82E009
:108210000E94CC0F0E94F80C0F5F1F4F802F8E1909
:10822000A82FB0E080917F0490E082959295907F96
:108230009827807F9827A817B907FCF21091450668
:108240008FE896E00E94E22C898389818F708F5F8E
:10825000809300041093C205898184FDB3C08CE033
:108260008093FF037AC9809104068093E806809189
:10827000BC05809329078091BE05809345068091B7
:108280004C0680934B0610924C068DCB992309F433
:108290004AC982E20E9436178DE00E94FE160E94B3
:1082A0000D191092840447C9939480918304981601
:1082B00008F412CE6624639416CE8091820420CCFA
:1082C00080918204EBCD0E94B415882309F017CA6F
:1082D00082E08093840413CA992D981B80918404B2
:1082E00080FFA1C0892F0E9404180ACDE92DF0E07B
:1082F000E751F94F80808EE00E948714882311F0A7
:10830000E0E18E2A8FE00E948714882311F0F0E2CA
:108310008F2A84E10E948714882311F080E8882A3C
:1083200085E10E948714882311F090E4892AE82DC2
:10833000F0E0EF73F070EE5FFB4F482D40788081E6
:1083400060E00E94871E82E0809384047092820421
:108350000E943215882309F444CD882E8A94EFE0D8
:108360008E228EE00E948714882311F0F0E18F2A7C
:108370008FE00E948714882311F080E2882A84E12C
:108380000E948714882311F090E8892A85E10E94D1
:108390008714882311F0E0E48E2AE82DF0E0EF73D3
:1083A000F070EE5FFB4F482D4078808160E00E94C6
:1083B000871E82E0809384043092820412CD109252
:1083C000820445CC80E14CCFE92DF0E0E751F94F34
:1083D00080828EE00E948714882381F588248FE0B4
:1083E0000E948714882311F080E2882A84E10E9489
:1083F0008714882311F090E8892A85E10E94871468
:10840000882311F0E0E48E2A80E00E949E1E93945F
:10841000FFE3F91518F410928304992470928404F0
:1084200010928204F5CD892F0E94D01769CC81E08B
:108430008093CF06809348060C94673890E1892E8C
:10844000CECF80E172CA84E00E94FE1679CC83E030
:108450000E94FE1675CC0F931F93CF93DF93EC0110
:10846000442319F18B0150E070E020E030E0F90185
:10847000ED52F94F60816F706F5FD80190E0FE019F
:10848000E50FF11D80818D939F5F5F5F9617B8F3B5
:10849000760F2F5F3F4F005F1F4F241740F3872F4A
:1084A000DF91CF911F910F91089570E0872FDF9199
:1084B000CF911F910F910895BF92CF92DF92EF92CB
:1084C000FF920F931F93CF93DF936B01B42E44233E
:1084D00069F17C0110E000E0C0E0D0E0C7010E943B
:1084E000E22CFE01ED52F94F808320812F702F5F27
:1084F000D70190E08D91F601E10FF11D80839F5F20
:108500001F5F9217B8F3020F219680E190E0E80E0A
:10851000F91ECB1518F3802FDF91CF911F910F918A
:10852000FF90EF90DF90CF90BF90089500E0F3CFE1
:10853000CF92DF92EF92FF920F931F93DF93CF932F
:10854000CDB7DEB7C054D0400FB6F894DEBF0FBE33
:10855000CDBF109284041092820482E08093810443
:1085600040914B068FE896E06E010894C11CD11C27
:10857000B6010E945C42E82E809183048E1510F0B3
:108580001092830480914B068823C1F090E030E084
:10859000E32FF0E0ED52F94F20812F702F5F80E044
:1085A000E92FF0E0E35BF94F80838F5F9F5F8217D5
:1085B000B8F33F5F80914B06381750F30E944C167A
:1085C00080913607882309F40EC284E00E94422D70
:1085D000FF240E944C160E94F80C1091CF06133015
:1085E00099F0143009F46EC0113079F10E94602FB7
:1085F000882379F70E942F2F0E944C160E94F80CB6
:108600001091CF06133069F70E94482D882309F096
:108610009EC10E94BA2E882311F010928F040E94EE
:108620003215882319F3182F11500E94ED18812F4D
:108630000E94C4181093D006809136078823B1F6A3
:108640008091D0068093D706D1CF0E94482D8823F1
:1086500009F06BC10E944D2F86E10E94DC14882333
:1086600029F080918504882309F08AC187E10E945E
:10867000DC14882329F080918504882309F096C1B1
:108680008091CF06813011F010928F0480913607CF
:10869000882309F06CC10E948D2C882309F4A6CF91
:1086A00010928104C05CDF4F0FB6F894DEBF0FBE9E
:1086B000CDBFCF91DF911F910F91FF90EF90DF9091
:1086C000CF9008950E94482D882309F013C110E02F
:1086D00086E10E94DC14882309F0F5C087E10E943E
:1086E000DC14882309F0D8C086E10E94B3148823E3
:1086F00009F0CCC087E10E94B314882309F0C0C000
:1087000086E10E949D14882309F0A8C08EE00E9493
:108710009D14882339F08F2D809580719FEEF9226A
:10872000F82A12E08FE00E949D14882339F08F2DE3
:10873000809580729FEDF922F82A12E084E10E9470
:108740009D14882339F08F2D809580789FE7F9223A
:10875000F82A12E085E10E949D14882339F08F2DBC
:10876000809580749FEBF922F82A12E00E9432155E
:10877000282F882361F08F2D90E08F7090700D97D7
:1087800034F421502F7080EFF822F22A12E088E0B2
:108790000E949D14882309F449C08F2D90E08F70AA
:1087A00090700D970CF4E7C090EFF92200E010E014
:1087B00080918304F601E80FF11DF08240914B0691
:1087C000C6016FE876E00E942B42E82E81E080939C
:1087D00085040D301105B4F58F2D61E00E94571A04
:1087E00084E20E94FE160E94C217E0918304F0E02A
:1087F000E35BF94F80810E94D0170E940D19809190
:10880000CF06843011F010928F04809136078823B0
:1088100009F180918E04813009F0E8CE10928E0427
:108820000E948D2C882309F4E1CE3ACF123009F44E
:10883000DEC0113021F70F2D10E00F7010700D30D9
:10884000110554F28F2D60E00E94571A84E20E94B5
:108850003617C9CF81E00E94422DDBCF80E00E9415
:108860008714882309F452CF8091C1058093830433
:1088700080918304F601E80FF11DF08011E046CFEE
:1088800080E00E9436170E940D193ACF82E00E94C4
:1088900036170E940D192ECF809183046E2D70E043
:1088A00090E00197860F971F0E940C4D80938304E0
:1088B00080918304F601E80FF11DF08080E00E94B2
:1088C000FE1611E011CF809183048F5F80938304A3
:1088D000809183046E2D0E94EC4C909383048091D0
:1088E0008304F601E80FF11DF08082E00E94FE167D
:1088F00011E0F4CE0E94AD1782E20E94FE1681E0E4
:1089000080938F0481E20E94FE1680918504882363
:1089100009F465C082E00E941A1780918304F60171
:10892000E80FF11DF08011E0D3CE0E94AD1782E276
:108930000E94FE1610938F0481E20E9436178091E8
:108940008504882379F182E00E941A1783CE0E9461
:10895000AD1781E00E94620284E20E94FE168091BF
:10896000D0060E94C41881E080938F0452CE84E028
:108970000E94422D90CE8FE0F82E0FE010E018CF2D
:1089800082E00E9436178091E806609129074091A5
:10899000450620914B060FE816E00E943E301092EB
:1089A000850464CE82E00E94361754CE82E00E9495
:1089B00036178091E806609129074091450620917D
:1089C0004B060FE816E00E94C92F40914B06C801E4
:1089D000B6010E945C42E82E1092850451CE82E0DE
:1089E0000E9436179ACF81E00E94422DF1CD0F2DC3
:1089F00010E00F701070DCCE2F923F924F925F927A
:108A00006F927F928F929F92AF92BF92CF92DF929E
:108A1000EF92FF920F931F93DF93CF93CDB7DEB703
:108A2000C058D0400FB6F894DEBF0FBECDBF109235
:108A300084041092820482E08093810440914B066A
:108A4000B1E4CB2ED12CCC0EDD1E8FE896E0B60122
:108A50000E945C42B82E0E944C16809136078823F3
:108A600009F463C684E00E94422DAA2433245524CD
:108A7000442466246A947724222423944E01089483
:108A8000811C911C0E944C160E94F80C1091CF067C
:108A90001F30D1F0103108F08DC0133009F454C2EA
:108AA000143009F4A7C2113009F471C20E94602F7A
:108AB000882341F70E942F2F0E944C160E94F80C29
:108AC0001091CF061F3031F70E94482D882309F0FE
:108AD00018C30E94BA2E86E10E949D14882309F0D3
:108AE00007C389E00E949D14882309F0F9C28AE037
:108AF0000E949D14882309F0D0C286E10E94B3141D
:108B0000882309F0D7C289E00E94B314882309F0B2
:108B1000DAC28AE00E94B314882309F0DDC28DE036
:108B20000E949D14882329F080917F04882309F0F6
:108B300065C591E0A91609F495C4A2E0AA1609F446
:108B40008DC4B3E0AB1609F0B1CF20928504652D3A
:108B500070E0832D992787FD9095860F971F840DD0
:108B6000911D0E940C4D482EBB2099F020E030E072
:108B7000F601E20FF31F842D820F652D0E94EC4C4D
:108B8000D401A90FB11D8C9180832F5F3F4F2B150E
:108B900078F340914B06C6016FE876E00E942B42C5
:108BA00040914B068FE896E0B6010E945C42B82ED9
:108BB000AA247CCF113109F41BC1113108F480C003
:108BC000123109F073CF0E94482D882309F02DC47B
:108BD0000E94BA2E8CE00E949D14882309F01CC4C8
:108BE0008CE00E94B314882309F012C48EE00E9426
:108BF0009D14882309F002C48FE00E949D148823ED
:108C000009F0F2C384E10E949D14882309F0E2C3B5
:108C100085E10E949D14882309F0D2C388E00E9458
:108C20009D14882309F0C2C38EE00E94B3148823E8
:108C300009F05EC38FE00E94B314882309F04BC390
:108C400084E10E94B314882309F04EC385E10E9499
:108C5000B314882309F00AC388E00E94B314882360
:108C600009F00DC3AA2009F421CF20928504BB206E
:108C700009F48FCF860110C00E97F9F08F2D862151
:108C8000D8019C919721892BF80181938F018E2F18
:108C90008C198B1508F07DCF0E941B01F82E90E0F7
:108CA0008F7090708D30910539F7E7EFFE228F2D90
:108CB00090E08F7090700E9709F7F7EFFF22DECFEC
:108CC0000E94482D882309F06BC30E94BA2E8CE0C5
:108CD0000E949D14882309F05DC387E10E949D14C2
:108CE000882309F051C380E00E949D14882309F075
:108CF00045C38CE00E94B314882309F03BC387E18D
:108D00000E94B314882309F031C380E00E94B31499
:108D1000882309F027C38EE00E949D14882309F060
:108D200017C38FE00E949D14882309F007C384E1D4
:108D30000E949D14882309F0F7C285E10E949D14CA
:108D4000882309F0E7C288E00E949D14882309F077
:108D5000D7C28EE00E94B314882309F0CDC28FE001
:108D60000E94B314882309F047C284E10E94B3141F
:108D7000882309F03DC285E10E94B314882309F0DD
:108D800033C288E00E94B314882309F029C2AA20C4
:108D900009F48CCE20928504E2E0AE1609F4BEC33D
:108DA000F4E0AF1609F476C4B1E0AB1609F033C4B1
:108DB000BB2009F4EECE860107C00F5F1F4F802F46
:108DC0008C198B1508F0E5CE0E941B01F82EEFE1FF
:108DD000E81798F30E941B01D8012C916B2D0E947B
:108DE000EC4CF601E90FF11D80818C932083E5CFD7
:108DF0000E94482D882309F02CC30E94BA2E8CE0D3
:108E00000E949D14882309F0E2C18CE00E94B314F3
:108E1000882309F0D8C18EE00E949D14882309F0B0
:108E2000C8C18FE00E949D14882309F0B8C184E175
:108E30000E949D14882309F0A8C185E10E949D1419
:108E4000882309F098C188E00E949D14882309F0C6
:108E500088C18EE00E94B314882309F05AC18FE0C4
:108E60000E94B314882309F05DC184E10E94B31409
:108E7000882309F060C185E10E94B314882309F0BA
:108E800063C188E00E94B314882309F066C18DE0B5
:108E90000E949D14882329F080917F04882309F083
:108EA00043C01A2D10FF02CE2092850411FDF6C298
:108EB000BB2041F1860106C00F5F1F4F802F8C1928
:108EC0008B1500F50E941B01F82EBFE3B817A0F325
:108ED0000E941B01F82E90E08F7090708D309105EC
:108EE00009F40BC30E9709F405C39F2D9621D801F1
:108EF0008C918721982B9C930F5F1F4F802F8C198B
:108F00008B1500F3BEEFAB2240914B06C6016FE814
:108F100076E00E942B4240914B068FE896E0B60126
:108F20000E945C42B82EC2CD8A2D80958270B1E03D
:108F3000AB22A82A8DE00E9436171A2DA1FCD2C3BD
:108F400055240E940D19AECF0E94482D882309F0A8
:108F500071C20E94BA2E882311F010928F040E94D1
:108F60003215A82E882309F4A1CDAA940E94ED18E9
:108F70008A2D0E94C418A092D006809136078823BB
:108F800009F094CD8091D0068093D7068FCD0E94B2
:108F9000482D882309F07BC10E944D2F8091CF0678
:108FA000813011F010928F0480913607882309F0E8
:108FB0006AC10E948D2C882309F478CD1092810417
:108FC000C058DF4F0FB6F894DEBF0FBECDBFCF91B4
:108FD000DF911F910F91FF90EF90DF90CF90BF90A6
:108FE000AF909F908F907F906F905F904F903F9049
:108FF0002F9008950E94482D882309F021C184E014
:109000000E94DC14882309F014C185E00E94DC145E
:10901000882309F007C182E10E94DC14882309F04B
:10902000FAC081E10E94DC14882309F0EDC00E949F
:109030004D2F86E10E94DC14882329F0809185045D
:10904000882309F0A8C287E10E94DC14882329F054
:1090500080918504882309F0B8C28091CF068430BE
:1090600051F010928F0482E00E94361782E20E9433
:1090700036170E94C21780913607882309F4C0C0B2
:1090800080918E04813009F011CD10928E040E94DF
:109090008D2C882309F40ACD91CF8CE10E94FE1615
:1090A000AF2CA3943324339486E10E94B314882315
:1090B00009F429CD82E00E94361789E00E94B3149A
:1090C000882309F426CD8BE10E9436178AE00E949E
:1090D000B314882309F423CD8CE10E9436171FCDE9
:1090E0008BE10E94FE16AF2CA39433243A94FFCC5C
:1090F00082E00E94FE163090C1053194AA24A39408
:10910000F0CC80E20E94FE16AA243324FF244424DB
:10911000E0CC84E00E9436178FE00E94B3148823CD
:1091200009F4A3CE83E00E94361784E10E94B314B1
:10913000882309F4A0CE88E00E94361785E10E94BA
:10914000B314882309F49DCE81E00E94361788E08D
:109150000E94B314882309F49ACE84E20E94361741
:1091600096CE84E20E94FE16A1E0AA2A1FE0612E9C
:10917000B0EF7B2E6ECE81E00E94FE1691E0A92A10
:1091800080E4682E0FEB702E5ECE88E00E94FE1603
:1091900081E0A82A20E8622E9FE7792E4ECE83E058
:1091A0000E94FE16F1E0AF2A40E2642E3FED732EDE
:1091B0003ECE84E00E94FE16E1E0AE2A60E1662E1B
:1091C0005FEE752E2ECE8EE00E94361724CE8EE0F6
:1091D0000E94FE16B1E0AB2A66246A94772415CE6D
:1091E00084E20E943617D3CD81E00E943617C9CDA4
:1091F00088E00E943617BFCD83E00E943617B5CDB8
:1092000081E00E94422D3CCF6091CF0681E141E197
:109210000E942E2D0CCF6091CF0682E142E10E9488
:109220002E2DFFCE6091CF0680E145E00E942E2DCD
:10923000F2CE6091CF068FE044E00E942E2DE5CE65
:109240000E94AD1782E20E94FE1620928F0481E2F6
:109250000E94FE1680918504882309F4AEC182E045
:109260000E941A1781E00E946202C9CE81E00E942A
:10927000361788E00E94B314882309F4F3CC84E203
:109280000E943617EFCC84E00E94422D92CE0E94BD
:10929000AD1782E20E94FE1610938F0481E20E94B5
:1092A00036178091450660914B064091BE0520918E
:1092B0004C0600914506E090BC050E94FC19809187
:1092C0008504882309F47DC182E00E941A1781E099
:1092D0000E94620261CE83E00E94361784E10E9400
:1092E000B314882309F4B2CC88E00E943617AECCC0
:1092F00084E00E9436179ECC84E00E9436172FCD62
:1093000084E20E94FE16F4E0AF2EEFE06E2E70EFC6
:10931000772E1FCD81E00E94FE1614E0A12EB0E44E
:109320006B2EAFEB7A2E0FCD88E00E94FE1694E0F4
:10933000A92E80E8682E0FE7702EFFCC83E00E94F4
:10934000FE1644E0A42E30E2632E2FED722EEFCCF9
:1093500084E00E94FE1674E0A72E60E1662E5FEEA8
:10936000752EDFCC82E20E943617D5CC80E00E94B9
:109370003617CBCC8EE00E943617C1CC82E20E9419
:10938000FE16E3E0AE2EB5CC80E00E94FE16F2E0C1
:10939000AF2EA9CC8EE00E94FE16AA24A3949DCCE9
:1093A00089E10E94FE16AA2433248FCC84E20E9415
:1093B000FE16AA24A3942FE0622E90EF792E34CCCF
:1093C00081E00E94FE16AA24A39440E4642E3FEBA1
:1093D000732E24CC88E00E94FE16AA24A39460E891
:1093E000662E5FE7752E14CC83E00E94FE16AA2439
:1093F000A394E0E26E2E7FED772E04CC84E00E94F1
:10940000FE16AA24A394A0E16A2EFFEE7F2EF4CBD1
:109410008EE00E943617EACB8EE00E94FE16AA2448
:10942000A39466246A947724DBCB8BE00E94FE161B
:10943000AA24CECB0E94AD1781E00E94620284E292
:109440000E94FE168091D0060E94C41820928F04BC
:1094500080CD8CE00E94FE16AA24CFCC332009F0E8
:1094600074CB24CB332009F421CBA0928504BB20FC
:1094700089F0332D3B0DD60120E0822F830F6B2D19
:109480000E94EC4CF401E90FF11D8D9180832F5F58
:109490002B1598F340914B06C4017ECBBB2009F4F9
:1094A00031CD860107C00F5F1F4F802F8C198B15A0
:1094B00008F028CD0E941B01F82EEFE3E81798F37F
:1094C0000E941B01652D0E94EC4CF401E90FF11D77
:1094D000F0808F2D90E08F7090708D309105B9F0F5
:1094E0000E9791F09F2D9621D8018C918721982B72
:1094F0009C93D9CFF7EFFF22F8CCE7EFFE228F2D18
:1095000090E08F709070EECC87EFF822EBCFF7EF02
:10951000FF228F2D90E08F709070E2CF6B2D6695BB
:10952000D9F09B2D915040E050E0A92FB0E094017C
:10953000240F351FF601EA0FFB1F8081F90180839C
:10954000A80DB91DF601E40FF51F80818C93915091
:109550004F5F5F4F461748F3BB2009F41ACB81E0F9
:1095600040E050E06B2D0E94EC4CD601A40FB51FDB
:10957000F401E90FF11D20812074F401E40FF51FBF
:1095800080818F7B282B2C93892F8F5F4F5F5F4FBC
:109590004B1540F3FECA82E00E9436178091E80620
:1095A000609129074091450620914B060FE816E08F
:1095B0000E943E301092850446CD82E00E9436170C
:1095C00051CE82E00E94361782CE82E00E9436178A
:1095D0008091E806609129074091450620914B064D
:1095E0000FE816E00E94C92F40914B06C801B60152
:1095F0000E945C42B82E109285042FCDF39481E036
:10960000F8228DE00E943617FF2009F077C055241C
:109610000E940D198ECA60914B068FE896E0A60154
:1096200023EC35E00E94502DE82E882311F18601AD
:1096300006C00F5F1F4F802F8C198E15D0F40E942B
:109640001B01F82EBFE3B817A0F30E941B01F8011D
:1096500020816E2D0E94EC4CF601E90FF11D8081F6
:10966000D8018C9320830F5F1F4F802F8C198E158C
:1096700030F360914B068FE896E0A60123EC35E0CD
:109680000E94312E40914B068FE896E0B6010E9471
:109690005C427FCABB2009F47CCA860107C00F5F09
:1096A0001F4F802F8C198B1508F073CA0E941B0165
:1096B000F82E8FE38F1598F30E941B01D8012C918F
:1096C0006B2D0E94EC4CF601E90FF11D8081862183
:1096D000972D9223892B8C93808187212621822BA1
:1096E0008083DDCF8DE00E94FE1685E096E0B40118
:1096F00040917F040E945C42582E23CC8DE00E9452
:10970000FE1685E096E0B40140917F040E945C4221
:10971000582E40914B068FE896E0B6010E945C42BD
:10972000B82EA3E0AA2E332473CF81E00E94422DED
:109730009CC9EF920F931F930E944C16809136079D
:10974000882309F426C184E00E94422D07C011300D
:1097500009F47EC00E94602F8823E1F00E944C161D
:109760000E94F80C1091CF061330F1F0143078F30A
:10977000143009F447C01D3069F781E00E94A23619
:109780008091CF068D3031F310928F040E94602FAC
:10979000882321F70E942F2F0E944C160E94F80C5C
:1097A0001091CF06133011F70E94482D882309F03D
:1097B0009AC00E94BA2E882321F010928104109240
:1097C0008F040E943215882309F07AC080913607F1
:1097D000882309F0BFCF86E10E949D14882309F4F5
:1097E000B9CF80E00E949E1E81E00E94CC0F80E2F3
:1097F0000E94262D9091D706890F60E040E00E94DC
:10980000871EA8CF0E94482D882309F081C080E0E0
:109810000E94A236882309F478C08091CF06843054
:1098200011F010928F0480913607882309F48DC0BF
:1098300080918E04813009F08DCF10928E040E94A9
:109840008D2C882309F486CF1F910F91EF900895F6
:109850000E94482D882309F07CC080E00E94A23637
:10986000182F86E10E949D148823C9F41123A1F0CA
:109870008091CF06813011F010928F0480913607CD
:10988000882309F082C00E948D2C882309F462CFBE
:109890001F910F91EF9008950E944D2FE9CF80E026
:1098A0000E949E1E81E00E94CC0F80E20E94262D25
:1098B0009091D706890F60E040E00E94871ED6CFC6
:1098C000182F11500E94ED18812F0E94C418109378
:1098D000D00680913607882309F078CF8091D00692
:1098E0008093D70673CF0E94AD1711E010938104C7
:1098F00081E00E94620284E20E94FE168091D006FE
:109900000E94C41810938F0454CF0E944D2F85CF0E
:109910000E94AD1782E20E94FE1681E080938F04C0
:1099200081E20E94FE168091450660914B064091AF
:10993000BE0520914C0600914506E090BC050E94B2
:10994000FC1981E00E94620262CF81E00E94422DF8
:109950006FCF0E94AD1782E20E94FE1610938F0413
:1099600081E20E9436178091450660914B06409136
:10997000BE0520914C0600914506E090BC050E9472
:10998000FC1981E00E94620268CF84E00E94422DAF
:109990007ACF81E00E94422DE1CE629FD001739F79
:1099A000F001829FE00DF11D649FE00DF11D929F7B
:1099B000F00D839FF00D749FF00D659FF00D9927BA
:1099C000729FB00DE11DF91F639FB00DE11DF91FDE
:1099D000BD01CF0111240895991B79E004C0991F9E
:1099E000961708F0961B881F7A95C9F780950895F9
:1099F000AA1BBB1B51E107C0AA1FBB1FA617B707B5
:109A000010F0A61BB70B881F991F5A95A9F78095D0
:109A10009095BC01CD01089597FB092E07260AD029
:109A200077FD04D0E5DF06D000201AF4709561952B
:109A30007F4F0895F6F7909581959F4F0895A1E285
:109A40001A2EAA1BBB1BFD010DC0AA1FBB1FEE1FB8
:109A5000FF1FA217B307E407F50720F0A21BB30B03
:109A6000E40BF50B661F771F881F991F1A9469F77F
:109A700060957095809590959B01AC01BD01CF01DB
:069A80000895F894FFCFE9
:109A860001FFFFFFFFFFFFFFFFD012130000060CD0
:109A960012000A101A000100010001000100010075
:109AA600010001000100010001000100010001C0E8
:109AB60000800040007F206430480F04050607112F
:109AC6001210130E04050607111210130409050AD5
:109AD60006070B110C120D1013252123262724220D
:109AE600201D1E1B191F1C1A1012180F110C130E05
:109AF6000B140D0A151609170405080306010700BD
:109B0600020320191A180C0B0A0904080120191A55
:109B1600180C0B0A092221252320191A18241B1CAC
:109B26000F0E0D04030A0C0B0908010200201B1975
:109B36001C1A180F0C0E0B0D0A0926271D1E1F10C6
:109B4600121113141516170506076E306E78307845
:109B5600000100070E091C1B1215383F363124235D
:109B66002A2D70777E796C6B6265484F4641545357
:109B76005A5DE0E7EEE9FCFBF2F5D8DFD6D1C4C3C7
:109B8600CACD90979E998C8B8285A8AFA6A1B4B3B7
:109B9600BABDC7C0C9CEDBDCD5D2FFF8F1F6E3E427
:109BA600EDEAB7B0B9BEABACA5A28F888186939417
:109BB6009D9A2720292E3B3C35321F181116030487
:109BC6000D0A5750595E4B4C45426F686166737477
:109BD6007D7A898E878095929B9CB1B6BFB8ADAAD7
:109BE600A3A4F9FEF7F0E5E2EBECC1C6CFC8DDDAD7
:109BF600D3D4696E676075727B7C51565F584D4A47
:109C06004344191E171005020B0C21262F283D3A36
:109C160033344E49404752555C5B7671787F6A6DA6
:109C260064633E39303722252C2B0601080F1A1D96
:109C36001413AEA9A0A7B2B5BCBB9691989F8A8D06
:109C46008483DED9D0D7C2C5CCCBE6E1E8EFFAFDF6
:109C5600F4F30409050A06070B110C120D10130084
:109C660001000100010001000100010001000100E6
:109C7600010001000100010001C000800040000C4D
:109C860001011718191A1B1C1D1E1F202122233F14
:109C96003F3F0B0C0D0E0F10111213141516173F24
:109CA6003F3F232425262728292A2B2C2D2E2F3FDC
:109CB6003F3F0B0C0D0E0F10111213141516173F04
:049CC6003F3F150007
:00000001FF
